:10709E00383838003631320020202000535350004B
:1070AE005545530041555300554550005349430033
:1070BE0039393900524553004144520043202000D3
:1070CE002D2D2D004552520053434E004141460096
:1070DE00412020004520200043203200434820005C
:1070EE00432031004C2020004F2020005020200053
:1070FE005553450000000000000000000000000095
:10710E000000000000000000000000000000000071
:10711E000000000000000000000000000000000061
:10712E00000800003F065B4F666D7D077F6F000015
:10713E000000000000777C395E79713D76301E00CC
:10714E001800545C7300506D003E000000000001FA
:10715E0002040810204080400408105C000000006B
:10716E00000003060A0F14191E23282D323C465028
:10717E005F010204081020408000FEFDFBF7EFDFE8
:10718E00BF7F0003130411021200100100408000A3
:10719E0000090012000900000101030000000000B8
:1071AE0000000000010001020203000000000000C8
:1071BE0000000000000000000000000004000100BC
:1071CE0000000000000000000800000800000000A1
:0371DE00000000AE
:1071E100013704017901017F20018400C193C1317C
:0871F100C1AB012800012B00D5
:10010000C2AFE4F5A8F5E8C28C438901758CFD7592
:100110008A65D28CF5B8F5F8D2BBD2B8D2A9C28D17
:10012000C28FD2ADD288C289C2B6D2AFF570757215
:1001300001753C097559097538FF7555FF7533010F
:10014000780F7405F2D22EC228C220C2B3D2B4C234
:10015000B5C2B47F647E00125FD0D2B4E531D394CF
:10016000054003C38001D39227E4789AF678A3F67A
:10017000789BF678A4F6789CF678A5F6202762FF9F
:1001800012565FE4FF1256BC7FFFC23A1257557BEE
:10019000057A70799EE4FD12540E78B276DF78B05D
:1001A00076DF78A076DF789E76DF78B3762078B138
:1001B000762078A17620789F7620788276DF788006
:1001C00076DF787C76DF787A76DF788376207881C0
:1001D0007620787D7620787B76207FF47E01125F12
:1001E000D020275D1257377B057A7079A2E4FD1283
:1001F000540EE4FF12565F12584778B376DF78B199
:1002000076DF78A176DF789F76DF78B2762078B0D7
:10021000762078A07620789E7620788376DF7881A5
:1002200076DF787D76DF787B76DF7882762078805F
:100230007620787C7620787A76207FF47E01125FB3
:10024000D07F097D857B0212735E50F57886E66467
:100250001C700418E66402604AE4F556F555E5554D
:100260002430FF7D567B011272F050F20555E555A2
:10027000D3940F40E9E4F556F555E5552450FF7D3C
:10028000567B011272F050F20555E555D3940F409C
:10029000E97885760208761C7F097D857B021272DB
:1002A000F050F57B057A7079A6E4FD12540E7FFFBD
:1002B000125783E4FF12565FE4FF1256BC125847F0
:1002C0007F067D857B0312735E7885E6B45A0A0843
:1002D000E6B4410508E6786DF2202709786DE2FF63
:1002E0007E00125FD0125FF4787FE62405798FF7E5
:1002F0007890760108760B7533FF20272675301924
:10030000E533B4FF141530E530600EC23A12606276
:100310007FC87E00125FD080E7E533F47039753313
:100320000180347570FF753064D2A8C2021260ACCF
:100330007F0A7E00125FD0303603D530EE7F0A7E12
:1003400000125FD0E533B4FF03D530F1E533B4FFDD
:1003500003753301E4F5707F2B7D3A7B0112735EE8
:100360005007E53AD394094003E4F53A7F3B7D58C2
:100370007B0112735E5007E558D394094003E4F5FE
:10038000587F207D057B0A1273A37F307D1D7B0A79
:100390001273A37F407D2F7B0A1273A37F507D567B
:1003A0007B0A1273A3741D2558F8E2F55A740525CB
:1003B0003AF8E2F53D74562558F8E2F55E54E0FF50
:1003C000BF2002155A20276C787FE62407798FF723
:1003D000E53D5407FFC43354E044057890F67805B2
:1003E000E27891F67806E27892F67807E27893F66A
:1003F0007808E27894F67809E27895F675650AC28D
:100400003B1260144003D565F6780AE27891F678DD
:100410000BE27892F6780CE27893F6780DE2789415
:10042000F6780EE27895F675650AC23B12601440C4
:1004300003D565F67F027D657B0112735E5031E561
:100440006530E002D21BE56530E114E53D6010F552
:100450006A786CF2E4F5727570054339018011E534
:100460006520E10CAF5AE55E54E0FD12374DD21B1A
:100470007F037D657B0112735E5011E565C39409AE
:10048000500AE565D39400400385653C7F047D6593
:100490007B0112735E5011E565C39409500AE5654E
:1004A000D3940040038565597802740AF208741EDB
:1004B000F2087428F278007405F2F565E4783AF2EF
:1004C000780174C8F278547409F2087460F2E53364
:1004D00090719D93F556E4F530301AFDC21A7802FA
:1004E000E214F27025740AF27804E214F2700574D2
:1004F00028F2B21F7803E214F2700F741EF27FFF2D
:100500001257A2788406E65403F67800E2700302DC
:1005100005EE14F260030205EE3027047F648002CA
:100520007F327800EFF21211D912269F20270A128B
:1005300072DEEF30E703125FF430270320360E122D
:100540000868500978547409F2087460F230144A4B
:10055000C214E5706401600BE57070377813E264D3
:10056000017030E54C54C0602AE54C543FFAE54D2B
:10057000FB7C007D64FFAE02127B3FAF05C0077CB1
:10058000007D64AF03AE02127B3FAD07D00712526D
:10059000AD8007AF6AAD301252AD302305C22312D1
:1005A0003ED0302A05C22A12497B302C05C22C12BB
:1005B0004253300505C205124DAC300B05C20B127B
:1005C0004A12300F05C20F125095301005C210129A
:1005D0004EC7300905C209124F8A3027030206614F
:1005E000783AE204F2543F70784339408073E57002
:1005F0009071A59320E00B7F06E4FDC23A1258BE2D
:10060000805F7800E2640A7058201B0578A2E670CB
:1006100050E53F540CFFBF0C167F06E540C3940223
:1006200050047D0280027D01C23A1258BE8032E53C
:100630003F540CFFBF08167F06E540C394085004E2
:100640007D0280027D01C23A1258BE80147F06E509
:1006500040C3941050047D0280027D01C23A1258BA
:10066000BE12516C303507C2351260C8C20A20274D
:1006700012E56560251565E565701F75650512084D
:10068000688017303614E5656010D5650DE58A542D
:100690000F2432F565C2021260AC7801E260591491
:1006A000F2705574C8F2120736302715785408E2F4
:1006B000FF24FFF218E2FE34FFF2EF4E7003120740
:1006C0000AE53F5430FF60307810E2602B14F2707E
:1006D00027E570B40122BF100E78687418F2781CF8
:1006E0007401F2D20C800A78687419F2781C7402D2
:1006F000F2753920E47810F2202D030204D9C22DBE
:0A07000043871075FF320204D9226E
:10070A00750E32D2B4150EE50E6020C293D294D281
:10071A0095D21C7F0A7E00125FD0C21CD293D2945B
:0C072A00D2957F0A7E00125FD080DA2298
:10073600780FE2600314F222302703020821E53124
:10074600C394055010C21DC2157F01E4FDC23A12C2
:1007560058BE12070A787EE6FFE571D39F4004A6CD
:10076600718014E5712401FDE433FCC3ED9F7480B0
:10077600F86C985002D231302E3730B413C2B47FA1
:1007860001E4FDC23A1258BE780F7402F202086202
:10079600788CE22402FFE433FEC3EF956B7480F895
:1007A6006E985003D38001C3921D9215C22E020883
:1007B6006220B439E56B2402FFE433FE788CE2D381
:1007C6009FEE6480F8748098402320311C7879E687
:1007D6006017787EE6D39464400F787916D22E7827
:1007E6000F7401F2D2B4020862C21D806FE57090E8
:1007F60071A59320E1667871E220E760301D0B7FDA
:10080600017D02C23A1258BE805220294F30154C43
:100816007F017D01C23A1258BE8041E56BD39493A5
:10082600500312070AE5709071A59320E1217871B3
:10083600E220E71BE56BD39497500B7F017D02D234
:100846003A1258BE80097F01E4FDC23A1258BEE54D
:1008560031D394054006C227D2B4D22E788CE56BEC
:02086600F2227C
:10086800301908C2011260970211C73027063036C6
:10087800030211C7E53930E522787FE62405798F30
:10088800F778907601781CE27891F6C23A126062A5
:1008980040030211D05339DF0211D0301E03021178
:1008A800C7302703020ACEE53920E603020960783B
:1008B8003AE2FF64407037787FE62407798FF7784B
:1008C8006DE25407FEC43354E044057890F6780589
:1008D800E27891F67806E27892F67807E27893F66D
:1008E8007808E27894F67809E27895F6805AEF6409
:1008F800807037787FE62407798FF7786DE25407A0
:10090800FFC43354E044057890F6780AE27891F60B
:10091800780BE27892F6780CE27893F6780DE27824
:1009280094F6780EE27895F6801EE570601A787F66
:10093800E62406798FF7786DE25407FFC43354E054
:1009480044017890F608A63DC23A1260624003025C
:1009580011D05339BF0211D07880E230E01D787F82
:10096800E62405798FF778907601087604C23A1262
:1009780060627880E254FEF20211D07880E230E1C1
:100988001D787FE62405798FF7789076010876053B
:10099800C23A1260627880E254FDF20211D0788087
:1009A800E230E22BE56C7002056C787FE62405796D
:1009B8008FF77890760308760608763FE56C14087A
:1009C800F6C23A1260627880E254FBF20211D078E3
:1009D80080E230E332787FE62405798FF7789076E5
:1009E80004087606E56C7005087652800C789276D5
:1009F80021E56C1408F608A673C23A126062788082
:100A0800E254F7F20211D07881E230E01D787FE6F7
:100A18002405798FF778907601087604C23A126037
:100A2800627881E254FEF20211D07881E230E11D51
:100A3800787FE62405798FF778907601087605C2E5
:100A48003A1260627881E254FDF20211D07881E2B4
:100A580030E329787FE62405798FF77890760508C2
:100A6800760608765508A66C08A67308A66EC23ADC
:100A78001260627881E254F7F20211D07860E230B5
:100A8800E044787FE62405798FF778907607087632
:100A980018788EE27892F67889E27893F6E408F688
:100AA80008F6E56C600414FF80027F007896A607BC
:100AB80008A673C23A12606240030211D07860E25D
:100AC80054FEF20211D07880E220E403020B6FE5B5
:100AD8007064317053E54C54C064C06023788F76DD
:100AE8004508760808761408A63D08761C08A63D31
:100AF8000876ECE56C1408F608A673E408F680217D
:100B0800788F764508760808761408A63D08761D7D
:100B180008A64C08A64D0876ECE56C1408F608A65D
:100B280073C23A1260628036E57064347030788F30
:100B3800764508760808761408F608761CE55A54AF
:100B48003F448008F6E55A25E0440C546C6470086C
:100B5800F6E5501408F608A673C23A126062788067
:100B6800E254EFF20211D0E53920E003020C66E509
:100B78007064056003020C66E530605CE572640130
:100B88007056788F7640786DE2FD5407FFC4335471
:100B9800E044047890F6E53075F064A4FFE56A7ADD
:100BA800002FFBEA35F044C0F54C08F6AF038F4D33
:100BB80008A607786CE27893F608A605E4786CF244
:100BC800C225C224F53DF530D23A126062400302D4
:100BD80011D05339FE0211D0E56A5407FFC43354CB
:100BE800E044057890F608A66A786CE27893F6787F
:100BF8006DE27894F6E4786CF2C225C224F530E50B
:100C08007224FE601D04703578927640E5565403D0
:100C180090719A937895F6787FE6788FF6E4F53DAB
:100C28008027AF6A125E89BFFFDE78927680E4780B
:100C380095F6787FE6788FF6E4F55A800CE4789597
:100C4800F6787FE6240A798FF7E4F54CF54DD23A29
:100C580012606240030211D05339FE0211D0E53907
:100C680030E13D787FE62402798FF7E53D5407FFB0
:100C7800C43354E044067890F608A63D08A63E081A
:100C8800A63F08A64008A64108A64ED23A126062BE
:100C980050035339FD2027030211D0C21E0211D080
:100CA800E53920E203020D35787FE62403798FF7D2
:100CB800E53D5407FFC43354E044087890F608A68D
:100CC8003D08A641E53390719D9330E30FE53DD390
:100CD800947F400808A64C08A64D801BE543540F96
:100CE800FFE542C454F04F7893F6E545540FFFE50D
:100CF80044C454F04F08F6E547540FFFE546C45482
:100D0800F04F7895F6E549540FFFE548C454F04F85
:100D180008F608A64A08A64BD23A12606250035356
:100D280039FB2027030211D0C21E0211D0E5393049
:100D3800E340E55A70055339F7C322787FE6240467
:100D4800798FF7E55A5407FFC43354E04404789088
:100D5800F608A65A08A65B08A65C08A65DD23A1251
:100D6800606250035339F72027030211D0C21E02D4
:100D780011D0E53930E441788F7634E56A5407FFBD
:100D8800C43354E0440408F608A66AE53F30E0049A
:100D98007F0280027F007892A607786DE27893F64A
:100DA800E408F6302702D20AC23A1260624003020F
:100DB80011D05339EF0211D0E53930E76F7853E29B
:100DC800146040047056E4FF7E0274142FF8E2FDAC
:100DD8006009AC060E748F2CF8A6050FBF08EBEE61
:100DE800C3940A5006748F2EF8E4F6787FE6240838
:100DF800798FF7E53D5407FFC43354E044087890F1
:100E0800F68019787FE6240E798FF7E53D5407FFC1
:100E1800C43354E044017890F608A63DC23A126003
:100E28006240030211D053397F0211D07880E2303A
:100E3800E529787FE6240D798FF77890760308A660
:100E48006408A65A08A662202703435E02D23A1213
:100E580060627880E254DFF20211D07880E230E6F6
:100E680020787FE6240D798FF77890760208A664BB
:100E780008A65AD23A1260627880E254BFF2021190
:100E8800D07880E230E732787FE6240D798FF778E2
:100E980090760408A66408A65A08A65DE55E30E0C8
:100EA800047F0080027F017894A607D23A1260621C
:100EB8007880E2547FF20211D07881E230E5297817
:100EC8007FE6240D798FF77890760308760408A6D4
:100ED8005A08A662202703435E02D23A126062785B
:100EE80081E254DFF20211D07881E230E620787F87
:100EF800E6240D798FF77890760208760408A65ACA
:100F0800D23A1260627881E254BFF20211D078813D
:100F1800E230E726787FE6240D798FF7789076041B
:100F280008760408A65A08A65DE408F6D23A1260C4
:100F3800627881E2547FF20211D0E53B30E33DE56F
:100F480070B41712788F76500876A40876507827F0
:100F5800E27892F68016788F761D08760478A1E2FA
:100F68007891F67893F6F418F67894F6C23A126007
:100F78006240030211D0533BF70211D0E53B30E247
:100F88003B788F761D7893E2B401047F0380027F5B
:100F9800027890A60778A1E27891F6E56C600414CF
:100FA800FF80027F007892A60708A673C23A1260F3
:100FB8006240030211D0533BFB0211D0E53B30E005
:100FC80037E57064146005E570B4160F788F7650B5
:100FD8000876217827E27891F6800D788F761908BF
:100FE800760178A1E27891F6C23A12606240030273
:100FF80011D0533BFE0211D0E53B30E151E570B40E
:10100800161F788F76500876047827E27891F6E4F0
:1010180008F67862E2047893F67892E27894F6809B
:101028001D788F761C7841E2FFC43354E04402787F
:1010380090F678A1E27891F67864E27892F6C23A6E
:1010480012606240030211D0533BFD0211D0E53B10
:1010580030E723788F761E08760278A1E27891F639
:101068007864E27892F6C23A12606240030211D0C4
:10107800533B7F0211D0E53B30E620788F761C0881
:10108800760278A1E27891F6087663C23A12606235
:1010980040030211D0533BBF0211D0E53B30E42D91
:1010A800788F76187841E2FFC43354E0440378908F
:1010B800F678A1E27891F67864E27892F6C23A126C
:1010C800606240030211D0533BEF0211D07860E216
:1010D80030E425787FE6240B798FF77890760178CD
:1010E800A1E27891F6D23A12606240030211D078F8
:1010F80060E254EFF20211D07860E230E52B787F9D
:10110800E6240C798FF77890760278A1E27891F648
:10111800788DE27892F6D23A12606240030211D0DA
:101128007860E254DFF20211D07842E230E02578AC
:101138008F7680087683E408F608A65A08A66075B4
:101148006001C23A12606240030211D07842E25450
:10115800FEF280747842E230E11CE55A4480788FD0
:10116800F60876A108A662C23A126062505A78421E
:10117800E254FDF280527842E230E219E55A4480A6
:10118800788FF60876C0D23A126062503B7842E215
:1011980054FBF280337842E230E322E55A44807807
:1011A8008FF608768308A66208A66C08A673C23A6A
:1011B80012606250137842E254F7F2800BC3227F28
:1011C80020C23A125755C3227F20C23A125755D32C
:0111D80022F4
:1011D90030270D7870E2FF30E30630E20312070A88
:1011E9007870E230E31508E230E110781CE264021D
:1011F90060097402F243392002265A7868E214B46D
:10120900070040030213C9901217F8282873021225
:101219002C0212750212D40212F202130202135E98
:1012290002139E7899E6600E167B057A7079AA7D7D
:101239000512540E800B7B057A7079AA7D0512542C
:101249000E78A3E630E30B781C7402F243392002CE
:10125900265A78A4E620E1030213C97899E66003C7
:101269000213C9781CF243392002265A7B057A7089
:1012790079AE7D0512540E78A3E630E34212571970
:10128900125737E5721460131460192402701CE4B4
:10129900FF12565FE4FF1256BC80107F01C23A125A
:1012A900575580077F02C23A1257557F101257834C
:1012B9007F04125783E4781CF243392002265A78B6
:1012C900A4E620E1030213C902265A7B057A707944
:1012D900B27D0512540E78A3E620E3030213C9E494
:1012E900781CF243392002265AE570D3940340034F
:1012F9000213C97570090213C97B057A7079B67D25
:101309000512540E78A3E630E342125719125737E3
:10131900E5721460131460192402701CE4FF12565C
:101329005FE4FF1256BC80107F01C23A1257558004
:10133900077F02C23A1257557F101257837F041252
:101349005783E4781CF243392002265A78A4E63000
:10135900E16E02265A30160D7B057A7079BA7D0541
:1013690012540E800B7B057A7079AA7D0512540EF2
:1013790078A3E630E30B781C7402F2433920022685
:101389005A78A4E630E1397899E67034781CF2434A
:10139900392002265A30160D7B057A7079BA7D05F7
:1013A90012540E800B7B057A7079B27D0512540EAA
:1013B90078A3E630E30AE4781CF243392002265A7E
:1013C900E570B43E00400302265A9013DAF8282843
:1013D9007302149402149A0214A30214AC0214BBEB
:1013E90002161402265A02265A02265A02180F0217
:1013F90014B502161402189F0218B502265A0218CB
:10140900B50216140218BE0218CC02265A02161486
:1014190002194D02196802197102265A02265A0246
:1014290016C10214C102158E021764021994021A18
:101439002C021A8402265A021A95021B1F021B6AE1
:10144900021B97021C0B021C78021C81021CC90298
:10145900265A021CD9021D5C021DF0021E47021EFB
:1014690093021F28021F71021FC902206D0220BCAE
:1014790002211B02235802236F022407022494022B
:1014890024E60225330225C0022610122869022605
:101499005A122A4E400302265A22122B5F40030297
:1014A900265A22122F53400302265A2212321A02B6
:1014B900265A85727002265AAF3F123A5E8F56E558
:1014C9005654037005533FF3801BE55630E108532A
:1014D9003FF3433F04800EE55630E009E53F540CE5
:1014E9007003433F041257191257377FFF1257836E
:1014F900D2147861E24401F2E540C4540FFFE536A5
:10150900C4540FFE6F601AEED39F40047F0A800215
:101519007F2878A2A607E540C3941050027646D2E8
:1015290008E55AB53D0EE53F54C07008E55E54E044
:101539007002F55AAF3DE4FD125E2B5003E4F555F8
:10154900202B0AAF3D125D35E4F538800FAF3D120F
:101559005C4F50047F0080027F0A8F38125D09407A
:101569000A125D1F923A7F401257557F01C23A1203
:10157900575575700178137401F2D223D22CC22009
:10158900D22802265AAF5E123A5E8F56E55E54E0C3
:10159900F50C1257191257377FFF125783D2147857
:1015A90061E24401F2E55AB53D0EE53F54C07008C9
:1015B900E55E54E07002F53DE55E54E0700CAF5A0B
:1015C900125CF2EFF46003E4F538AF5AAD0C125D2A
:1015D9009550047F0080027F0A8F55125E54400A9D
:1015E900125E73923A7F401257557868E264096037
:1015F90002D2237F02C23A125755757002781374CA
:1016090002F2D22AC228D22002265A7870E2FF308A
:10161900E20C30E00912282312266E02265A78A31A
:10162900E630E308E4FF12277C02265A78A4E63064
:10163900E617E57264016004E5727005AF6A125C31
:10164900F27F0112277CE4F53878A4E630E24630CF
:101659002743E539703F201E3C125C09EF700302F5
:10166900265A786CE56AF28F6AD21478297404F2E2
:10167900EFD3947F500302265AE53390719D93204E
:10168900E30302265A7B057A7079BEE4FD12540EF3
:10169900C21402265A7829E2600D14F27009C21B9D
:1016A900C217F572433901786DE2600302265A7850
:1016B90061E24404F202265A200706789916E66088
:1016C9000978A3E620E20302175EAF728F70EF1468
:1016D900601E24F4602424FE602024F9603B24EF7A
:1016E90060502425705F1227F4786BE2F556805E0E
:1016F9001227C5786BE2F55680547FFF1257831283
:101709005719125737D214D228C220753009757269
:101719000B75700B433B0180357FFF1257831257BE
:1017290019125737D220C228D214433B0175300908
:10173900801C7850E2FF655AFEF55AEF6EF2625A44
:101749007570298009E4F530F56AFF12277CC20E0D
:10175900C20702265A1232AD02265A125847788613
:10176900E25407640770411257191257377B057AFB
:101779007079C27D0112540EE53024F76003022608
:101789005AE56C6450600302265A757017856C6AB5
:10179900E56A54FC7827F2E56A5403786AF2D2289C
:1017A900C220433B0802265A78A3E6FF30E203022F
:1017B90016D378A5E6FE30E0067886E26401F2EEFB
:1017C90030E2067886E26402F2EF30E0067886E2DB
:1017D9006404F27886E230E0097F037D03C23A129D
:1017E90058BE7886E230E1097F047D03C23A125877
:1017F900BE7886E220E20302265A7F147D03C23AAC
:101809001258BE02265A200E0E7B057A7079C67DC3
:101819000212540E02265A7F10D23A125755200747
:1018290006789916E6600678A3E630E22EAF728F45
:1018390070BF02081227F443390880031227C5E54F
:101849003D7003533EF7E55A7003535BF7C20EC26E
:1018590007E4781CF243392002265A20070302269E
:101869005AE572B401187F01D23A125755123C2B2E
:10187900500302265A123FCE400302265A227F0203
:10188900D23A125755124769EF6401600302265A8A
:10189900D22A43390822D214D22375720D75700DDC
:1018A90078137404F2E47899F602265A122C4E4001
:1018B9000302265A22757212757012D214D223E4C9
:1018C9007899F678A3E630E308E4FF12277C02262C
:1018D9005A123C2B500302265A7872E2F50D700613
:1018E9007871E230E01B789906E6640A6003022603
:1018F9006DE50D6006FF125FC180027F081250720C
:1019090022789CE6F50D700518E630E01E7899E618
:10191900C3940A500FE50D6006FF125FC180027F74
:1019290008125072E47899F602265A78A4E620E162
:101939000302265AD20C781C7401F24339208570AF
:101949007202265AD220C22875721675701678133B
:101959007405F2D214E47899F6789CF202265A12A8
:101969002E41400302265A2278A3E620E2030226EA
:101979005A433B01786AE2FF7827E22FF56A7570CE
:10198900147F10125783D21402265A78A3E630E244
:101999000878807402F20216D37899E6601316E685
:1019A900600302265AAF50AE4F7D041253A202269D
:1019B9005A78A4E630E625E4F54FF550C228C2204E
:1019C900D232D230E4FF12565FE4FF1256BC7B05D7
:1019D9007A7079CAE4FD12540E02265A20300302A5
:1019E900265A7F10D23A1257557F4F1239ED78A3F4
:1019F900E620E30302265AE550454F700302265AB2
:101A0900D228C2201257191257377B057A7079CE1E
:101A1900E4FD12540EE4F573D23285506C75701FD3
:101A290002265A78A3E630E20878807402F2021698
:101A3900D37F73C23A1237F150077F10D23A125747
:101A49005578A3E630E3193032087880E24404F28D
:101A590080067880E24408F2D23275702002265A54
:0F1A690078A4E620E60302265A7899760A0550FB
:101A7800E5507002054F75701E0219C578A3E6205F
:101A8800E20302265A78807402F20216D378A3E69B
:101A980030E2097881E24402F20216D37899E660CE
:101AA8001216E6600302265AAF6CFE7D041253A29A
:101AB80002265A203023E4F56CC228C220D232D242
:101AC80030E4FF12565FE4FF1256BC7B057A70794A
:101AD800CAE4FD12540E02265A7F10D23A12575504
:101AE8007F6CC23A1237F178A3E620E30302265A44
:101AF800E56C700302265AD228C2201257191257D1
:101B0800377B057A7079CEE4FD12540EE4F573D272
:101B18003275702302265A78A3E630E2097881E20A
:101B28004402F20216D37F73C23A1237F150077F8C
:101B380010D23A12575578A3E630E31120320EC27C
:101B4800307881E24408F275702402265A78A4E6B7
:101B580020E60302265A7899760A056C75702202E7
:101B68001AC178A3E630E2097881E24402F202164B
:101B7800D330300C7899760A056C757022021AC138
:101B88007899E606FF7E007D041253A202265AE5E4
:101B98005A2420FFE43403FEE4FD1253A278A4E69D
:101BA80030E62AE55A04FF7D20125E2B7842E25483
:101BB800FBF27851E254FBF2E4F555FFFD12374D84
:101BC800500302265A7F0112277C02265A78A4E67F
:101BD80030E51F7842E254FBF27851E254FBF2E41C
:101BE800FFFD12374D500302265A7F0112277C024F
:101BF800265A78A3E620E30302265AE4FF12277C3C
:101C080002265AE55A75F00AA4FFE560540F7C00D5
:101C18002FFFEC35F0FEE4FD1253A2E4FF1256BC90
:101C2800125719123ED07FFF1257837F02D23A1201
:101C38005755AF5E123A5E8F56E55A04FF7D201263
:101C48005D9550047F0080027F0A8F55E55A75F034
:101C58000A842450F530757227757027D20B7813D3
:101C68007403F2C228D2207861E24401F202265AB3
:101C7800122D18400302265A22C228D22075514735
:101C8800755252E560540F2430F5537B047A00797D
:101C9800517D0112540E7B057A7079D27D0512545C
:101CA8000E7FFF125783782AE204F264326003023F
:101CB8001614F530F56AF55AF55EFF12277C0226F0
:101CC8005A757025E4782AF27842E24404F2022632
:101CD8005A782AE204F2640A702E08E2640170213C
:101CE800203011F55AF5607B057A7079C27D0112B2
:101CF800540E80147B057A7079D67D0112540E80BB
:101D080007E4782AF275702E782AE2D394285003D3
:101D180002265A2030107842E24401F2E4782AF28E
:101D280012282302265AE47899F6755138E55A752F
:101D3800F00A842430F552E55A75F00A84E5F02457
:101D480030F5537B047A007951E4FD12540E757016
:101D58002C02265A78A3E630E2030216D37899E6D5
:101D6800601316E6600302265AAF50AE4F7D041288
:101D780053A202265A78A4E630E625E4F54FF5503A
:101D8800C232C228C220D230E4FF12565FE4FF12EA
:101D980056BC7B057A7079CAE4FD12540E02265AA5
:101DA80020300302265A7F10D23A1257557F4F121D
:101DB80039ED78A3E620E30302265AC3E54F9402DF
:101DC800500302265AC228D2201257191257377BBD
:101DD800057A7079CEE4FD12540E85506CE4F573E3
:101DE800D23275702D02265A78A3E630E203021625
:101DF800D37F73C23A1237F150077F10D23A125785
:101E08005578A3E630E31D3032057562028003750C
:101E1800620175702EE4782AF2D2327842E24408E0
:101E2800F202265A78A4E620E60302265A78997622
:101E38000A0550E5507002054F75702C021D8A780E
:101E4800A3E630E2030216D3782AE204F2640A60B9
:101E580003021614755138E55A75F00A842430F5D2
:101E680052E55A75F00A84E5F02430F5537B047A7C
:101E78000079517D0112540E7B057A7079D27D0567
:101E880012540E7FFF12578302265A78A3E630E2D7
:101E9800030216D37899E6601216E6600302265A02
:101EA800AF6CFE7D041253A202265A78A4E630E6EF
:101EB80023E4F56CC228C220D232D230E4FF125695
:101EC8005FE4FF1256BC7B057A7079CAE4FD1254B0
:101ED8000E02265A20300302265A7F10D23A125791
:101EE800557F6CC23A1237F178A3E620E303022645
:101EF8005AE56C700302265A14700302265A8000B1
:101F0800D228C2201257191257377B057A7079CE1A
:101F1800E4FD12540EE4F573D23275703002265A7D
:101F280078A3E630E2030216D37F73C23A1237F180
:101F380050077F10D23A125755E4782AF278A3E670
:101F480030E31120320ED2327880E24410F27570FC
:101F58003102265A78A4E620E60302265A789976B2
:101F68000A056C75702F021EBC78A3E630E20302E6
:101F780016D378A4E630E60C7899760A056C757065
:101F88002F021EBC7F73C23A1237F140A5782AE2AD
:101F980004F2B4640D7B057A7079D27D0512540E73
:101FA800801F782AE2FFC3948040030216D3EFC350
:101FB8009460400302265AEF540F600302265A80A9
:101FC8008578A3E630E2030216D37899E660131603
:101FD800E6600302265AAF50AE4F7D041253A202A8
:101FE800265A78A4E630E625E4F54FF550C228C213
:101FF80020D232D230E4FF12565FE4FF1256BC7B87
:10200800057A7079CAE4FD12540E02265A2030036C
:1020180002265A7F10D23A1257557F4F1239ED785F
:10202800A3E620E30302265AE550700302265A1459
:10203800700302265A24F8700302265A24E8700313
:1020480002265A8000C228D2201257191257377B0D
:10205800057A7079CEE4FD12540EE4F573D2327528
:10206800703302265A78A3E630E2030216D37F7350
:10207800C23A1237F150077F10D23A125755E47816
:102088002AF278A3E630E31120320ED2327880E2C9
:102098004410F275703402265A78A4E620E603024A
:1020A800265A7899760A0550E5507002054F7570E2
:1020B80032021FF578A3E630E2030216D378A4E6CD
:1020C80030E6127899760A0550E5507002054F758A
:1020D8007032021FF57F73C23A1237F14099782A9D
:1020E800E204F2B4460D7B057A7079D27D0512546C
:1020F8000E8020782AE2FFC3948040030216D3EFB3
:10210800C39441400302265AEF540F600302265A33
:1021180002209378A3E6FF30E20878807402F20286
:1021280016D3782EE2640F60030221E678A4E63025
:10213800E6137899760A754F00755001756C01752C
:10214800701E0219C5EF20E3030221DFE530D394A6
:10215800005007E56CD3947F40427F10D23A125763
:1021680055125719125737E4782EF2757035E53045
:1021780075F064A47C00256CFFEC35F044C0F54F85
:102188008F50F573756C117880E24409F2D228C239
:1021980020D232C2307899760202265AE53070375A
:1021A800E56C60337F10D23A1257551257191257FF
:1021B80037782E7405F2757035856C73754F008508
:1021C8006C50756C017880E24409F2D228C220D2A2
:1021D80032C230789976027F6CD23A1237F1789908
:1021E800E6700302265A16E6600302265A7602783B
:1021F8002EE2B40F00400302265A902209F828283C
:102208007302223602225C0222820222820222A861
:1022180002223602225C02225C0222E302223602F9
:10222800225C02228202230002225C02233B056D0B
:10223800E56DD394054003E4F56DE56D245BF55138
:102248007552207553207B047A007951E4FD1254AD
:102258000E02265A056DE56DD394054003E4F56D2D
:10226800755167E56D245BF5527553207B047A0040
:102278007951E4FD12540E02265A056DE56DD3948A
:10228800054003E4F56D755167755267E56D245B8C
:10229800F5537B047A007951E4FD12540E02265A54
:1022A800E54F543FFAAB507C007D64AF03FE127BD0
:1022B8003FAF05C0077C007D64AF03AE02127B3FD1
:1022C800AD07D0071252AD7F10C23A125755E4F548
:1022D8006CF530782E740FF202265AAF507E00E467
:1022E800FD1253A27F10C23A125755E4F56CF5302F
:1022F800782E740FF202265A7F10C23A125755E50B
:102308004F543FFAAB507C007D64AF03FE127B3F15
:10231800AF05C0077C007D64AF03AE02127B3FAD02
:1023280007D0071252ADE4F56CF530782E740FF231
:1023380002265A7F10C23A125755AF737E00E4FD49
:102348001253A2E4F56CF530782E740FF202265A77
:10235800AF6A125CF2E4FF1236FA40057F011227D9
:102368007CE4F53802265A782AE204F2640A703CC2
:10237800782DE2D394015034203014E478A1F2434C
:102388003B087B057A7079C27D0112540E801D7856
:102398002DE2B4010D7B057A7079D67D0112540EB9
:1023A800800AE478A1F2782AF275703A2030107821
:1023B8002AE2D394644008E4F212282302265A2021
:1023C800300302265A782AE2D39428500302265A68
:1023D800E47899F675513978A1E2FF75F00A8424FA
:1023E80030F552EF75F00A84E5F02430F5537B049C
:1023F8007A007951E4FD12540E75703802265A7825
:10240800A3E630E2030216D37899E6601216E66076
:102418000302265AAF6CFE7D041253A202265A7894
:10242800A4E630E623756C01D232C228C220D2302D
:10243800E4FF12565FE4FF1256BC7B057A7079CA36
:10244800E4FD12540E02265A20300302265A7F1049
:10245800D23A1257557F6CC23A1237F178A3E62068
:10246800E30302265AE56C700302265AD228C220DA
:102478001257191257377B057A7079CEE4FD12543A
:102488000EE4F573D23275703902265A78A3E63015
:10249800E2030216D37F73C23A1237F150077F1056
:1024A800D23A12575578A3E630E31E3032077893B4
:1024B8007402F2800578937401F275703AE4782A10
:1024C800F2D232433B0402265A78A4E620E60302FD
:1024D800265A78997605056C75703802243078A3E9
:1024E800E630E2030216D3782AE204F2640A6003B3
:1024F80002161475513978A1E2FF75F00A84243068
:10250800F552EF75F00A84E5F02430F5537B047A30
:102518000079517D0112540E7B057A7079D27D05C0
:1025280012540E7FFF12578302265A78A3E630E230
:10253800030216D37899E6601216E6600302265A5B
:10254800AF6CFE7D041253A202265A78A4E630E648
:1025580023756C01D232C228C220D230E4FF125651
:102568005FE4FF1256BC7B057A7079CAE4FD125409
:102578000E02265A20300302265A7F10D23A1257EA
:10258800557F6CC23A1237F178A3E620E30302269E
:102598005AE56C700302265AD228C2201257191223
:1025A80057377B057A7079CEE4FD12540EE4F57343
:1025B800D23275703C02265A78A3E630E20302163E
:1025C800D37F73C23A1237F150077F10D23A1257AD
:1025D8005578A3E630E31F303206E47889F28005A7
:1025E80078897401F275703DE4782AF2D232786005
:1025F800E24401F2805C78A4E630E65678997605E4
:10260800056C75703B02255C78A3E630E203021680
:10261800D3782AE204F2640A600302161475513171
:10262800788EE2FF75F00A842430F552EF75F00ACF
:1026380084E5F02430F5537B047A0079517D01124A
:10264800540E7B057A7079D27D0512540E7FFF12E5
:102658005783E4789AF678A3F6789BF678A4F67808
:062668009CF678A5F622A5
:10266E00C21EC219E4783BF2F5397852F2F53B18E6
:10267E00F27842F27885F27880F27887F27881F2F9
:10268E007865F27860F2C236F577C2B6D2A8C28EFD
:01269E002219
:10269F00201E0302275B7867E204F2D3941E405D8D
:1026AF00E5709071A59320E20D7B057A7079DA7D44
:1026BF000512540ED221C21E783BE242397852E203
:1026CF00423B7842E2FF7851E2FEEF4E7842F278D9
:1026DF0080E2FF7885E2FEEF4E7880F208E2FF7825
:1026EF0087E2FEEF4E7881F27860E2FF7865E2FED6
:1026FF00EF4E7860F2C219E47867F2C23620276C89
:10270F007867E254077065C21E783BE2423978520F
:10271F00E2423B7842E2FF7851E2FEEF4E7842F21E
:10272F007880E2FF7885E2FEEF4E7880F208E2FFD4
:10273F007887E2FEEF4E7881F27860E2FF7865E20B
:10274F00FEEF4E7860F27FC21272DB22302105C29B
:10275F0021D2142230270320360EE5709071A593F5
:0D276F0020E3057F20125783E47867F222F3
:10277C008F10123B9A123BA3123BC17FFF1257835F
:10278C00125847E4FF12565FE4FF1256BC12266E35
:10279C00E51020E008E56A7011E530700D7B057AD4
:1027AC007079A6E4FD12540E8002D214E4F572F591
:0927BC00707827F2D232D22222F9
:1027C5007FFF125783125D09400A125D1F923A7FFF
:1027D500401257557F01C23A1257551257191257D1
:0F27E50037D223D22CD214D228C220E4F53022CE
:1027F4007FFF125783125E54400A125E73923A7F2F
:10280400401257557F02C23A1257551257191257A0
:0F28140037D223D22AD214C228D220E4F53022A0
:102823007FFF1257837B057A7079DEE4FD12540E25
:10283300E4FF12565FE4FF1256BCC207C20ED22257
:10284300D232E4F56CC228C220786BE556F2782CBC
:10285300E530F2E4F530E53390719D93F5567570EC
:062863001A789976C822E4
:10286900C20AC21BC217D22BC228C220E4F57212B7
:1028790057191257377870E2FF30E20730E0041237
:1028890028232278A4E630E7097F027D6A123AB24A
:102899008F5678A4E630E4097F047D6A123AB28F34
:1028A9005678A3E620E3030229997FFF125783781C
:1028B90013E2B4010FE56A7004E53060077570052D
:1028C90043390122E5306409706BE56AC3945040CD
:1028D90032E56AD3945C502B7E007F087D007B0330
:1028E9007A007995127BBAE56A54FC7827F2E56A91
:1028F9005403786AF2786274FFF2757014D2144343
:102909003B012278A1E56AF27E007F087D007B0306
:102919007A007995127BBAE56AB46312786E7463AA
:10292900F2D22375700F433B01E47899F622757052
:102939000B433B0122E5306408600EE530C3945037
:10294900401FE530D3945650187866E2F560785008
:10295900E2F55A757025E4782AF27842E24404F2E5
:1029690022E530B40714E56A7003022A4D75701028
:1029790078A1F27860E24410F2227813E2640260EE
:1029890067E530700BE56A60077570054339012208
:1029990078A4E630E24C203225E55630E00BE56AB2
:1029A9007007E5307003022A4DE53390719D93203D
:1029B900E307E5306003022A4D757201801D20325C
:1029C90007E5306003022A4DAF3D1236FA400C7B11
:1029D900057A7079A6E4FD12540E22757005433903
:1029E900012278A4E630E535E53064087003022950
:1029F90052203211E530704CAF561236E7AD07AFB1
:102A09006A12374D22AF5AE55E54E0FD12374D4048
:102A1900337B057A7079A6E4FD12540E227871E2AF
:102A2900FF30E40930E30678A4E620E617E4FF1254
:102A3900565FE4FF1256BC7F6AD23A1237F150044E
:052A4900E47813F22205
:102A4E0078A3E630E30C786CE56AF2E4FF12277C9B
:102A5E00C32278A3E630E21C7B057A7079E2E4FDAE
:102A6E0012540E12586D757003E47828F2783C7487
:102A7E00C8F2C32278A4E6FF30E10CD20C781C74A5
:102A8E0001F2433920C322EF30E207E4FF1236FA97
:102A9E00C32278A4E630E5397827E26021123BA301
:102AAE007F01125783E4F5727570147827E2F56A88
:102ABE00D220C228753009D214433B01C322AF5A2B
:102ACE00E55E54E0FD12374D40057F0112277CC3B1
:102ADE0022301B4778A4E630E322C21B75701B75AB
:102AEE0072014339107861E24401F2E53F30E0248F
:102AFE0043398078537401F2C21780182027157855
:102B0E009906E6D39432400CE4F6C21B757005F5B7
:102B1E0072433901123BD55036C32230171CE53FA4
:102B2E0030E01778A4E630E30A4339807853740115
:102B3E00F2C217D214123BD5C322123BD55002C398
:102B4E0022123C2B5002C322123FCE5002D322C37C
:012B5E002254
:102B5F0078A3E630E30C786CE56AF2E4FF12277C89
:102B6F00C32278A4E630E50FE4FFFD12374D400590
:102B7F007F0112277CC32278A4E630E20EAF3D120C
:102B8F0036FA40057F0112277CC32278A4E630E194
:102B9F000CD20C781C7401F2433920C32278A3E6BF
:102BAF0030E21C7B057A7079E2E4FD12540E125864
:102BBF006D757003E47828F2783C74C8F2C3221262
:102BCF003BD55002C322123C2B5002C3221247693D
:102BDF00EF64017063E55E30E63A30E01F7869E23A
:102BEF00FE90717F93555C600AEE25E0044408F572
:102BFF00628019EE25E04408F56280107869E2F5ED
:102C0F006290717F93555C60034362087880E24461
:102C1F0020F2D322E55E30E7187869E2F562907111
:102C2F007F93555C60034362087881E24420F2D3BE
:0F2C3F0022D22A433908D322BF0202D322C32252
:102C4E00C220D22878A3E630E31BE570B40F0FE460
:102C5E00FF12277C78A17463F2433B40C322E4FF4A
:102C6E0012277CC322123C2B5002C322789CE6F51D
:102C7E000F60237899E6C3940A4004E4F6C322E475
:102C8E00F50EE50F20E008C313F50F050E80F3AF28
:102C9E000E124E6AC3227872E2F50F601E78990604
:102CAE00E6B40A15E4F50EE50F20E008C313F50FA0
:102CBE00050E80F3AF0E124E6AD32278A4E630E1F1
:102CCE000F857072D20C781C7401F2433920C32226
:102CDE00E570B40F02C32278A3E630E21E757003CE
:102CEE007B057A7079E2E4FD12540E12586DE47889
:102CFE0028F2783C74C8F2C205C32278A4E630E20A
:0A2D0E0007AF3D1236FAC322C322BC
:102D180078A3E630E31A753008AF5A786CEFF2F50D
:102D28006A7850F27866E560F2E4FF12277CC322E5
:102D380078A4E630E541E560540F04F50E146020F0
:102D480014601D24FE600904700EE56054C0701004
:102D5800E56054C064806008E4FFFD12374DC3226B
:102D6800AF0E7866EFF2F560757025E4782AF27890
:102D780042E24404F2C32278A4E630E20EAF3D12E8
:102D880036FA40057F0112277CC32278A4E630E199
:102D98000CD20C781C7401F2433920C32278A3E6C4
:102DA80030E21F7B057A7079E2E4FD12540E125866
:102DB8006D125737757003E47828F2783C74C8F2BE
:102DC800C322123BD55002C322123C2B5002C3220D
:102DD800124769EF6401705FE560540F1475F008DD
:102DE800A4FF7869E2FE2FF562EE90718893FF5296
:102DF80063E56020E71BE56225E0F5620562E2EF26
:102E0800525FEE90717F93FF555C7008EF425F80D0
:102E180003855C5FE56030E60674082562F5627834
:102E280069E290717F93555C6003436240D20B78EE
:092E380042E24402F2D322C3225B
:102E410078A3E630E307E4FF12277CC32278A4E6E7
:102E510030E20EAF3D1236FA40057F0112277CC3E6
:102E6100227870E2FF30E20830E005122823C32205
:102E7100123C2B5002C322789CE6FF600F7899E642
:102E81007004789CEFF2E47899F6C322789CE2FF13
:102E91006044302703789906789906E6640A70360B
:102EA1007892F27899F6786AE2FE33333354F8F582
:102EB1000EEF20E007C313FF050E80F57899E50EAC
:102EC100F27862E50EF2D20F789A7401F2433B0276
:102ED100E4789CF2C32278A5E6FF6021E47899F6B4
:102EE100EE7002C322EE6F6006E4789CF2C3227892
:102EF100927404F27874F27899760A80A978A4E63B
:102F0100FE30E534786AE2045403F50EE4FF74956B
:102F1100250EF8E2700EEFC394045008050E530E0F
:102F2100030F80EA786AE50EF27827E2250EF56A4A
:102F3100D20FE47899F6C322EE30E114857072D293
:102F41000C781C7401F2433920E4789CF27899F6EC
:022F5100C32299
:102F53007870E2FF20E20302311B78A3E630E2033C
:102F630002311BEF30E005122823C3227871E230CF
:102F7300E243E55630E03EE572640170387FFF12AC
:102F830057837B057A7079E6E4FD12540EE4FF1251
:102F9300565FE4FF1256BC75702F786BE556F278D6
:102FA3002CE530F2756C02C228C220D232D230E452
:102FB3007899F6C3227871E230E546E55630E04170
:102FC300E5726402703B7FFF1257837B057A707949
:102FD300E6E4FD12540EE4FF12565FE4FF1256BC02
:102FE300757032786BE556F2782CE530F2754F0048
:102FF300755002C228C220D232D230E47899F6C387
:1030030022E5726401600302311978A5E6FF30E21C
:103013000F633E02D223783C7401F2433902C32288
:10302300EF30E50F633E04D223783C7401F2433959
:1030330002C32278A4E630E4267B057A7079EA7D20
:103043000112540E75700AE4F540D22378A2F643B8
:1030530039027811F278997632783C04F2C32278F7
:10306300A4E630E70F78A2E6700AB218D223783CC0
:1030730004F2C3227871E220E103023119E4FFFD77
:10308300C23A1258BE7F10E4FDC23A1258BE7F0105
:10309300E4FDC23A1258BEE55654037005533FF39C
:1030A300803EE55630E108533FF3433F048031E56A
:1030B3005630E02C78A5E6FF30E609533FF3433F53
:1030C30004433902EF30E709533FF3433F084339E1
:1030D3000278A4E630E009533FF3433F0C4339023F
:1030E300E53F540C24F8601324FC601A2408701F75
:1030F300E4FF7D01C23A1258BE80147F107D01C2E5
:103103003A1258BE80097F017D01C23A1258BE7837
:103113003C7401F2C322C322783CE214F2600678C5
:10312300A3E630E25FAF728F70BF0204D22A80241D
:10313300E570B40104D22C801BE570B427087572C6
:1031430026757026C322E570B40D0975720B757070
:103153000B433B017828E2FFB4030AE548600643CA
:103163003E02433902EFB4060AE5496006433E04D2
:103173004339027F0412578312571912586DD21420
:10318300D223C322301B18E572B40113F5707F04F8
:1031930012578312571912586DD214D223C3221215
:1031A3003C2B5002C322124285506AE572B40217C7
:1031B300E55E30E6087880E24480F28053E55E20E5
:1031C300E74E4339088049E572B401167828E2FFD7
:1031D300640B6004EFB40C054339028033433904B4
:1031E300802EE57264277028E56030E7047F4A800B
:1031F300027F488F6CE560540F256CF56CE5602009
:10320300E602156C855D737842E24408F27562014B
:07321300783C74C8F2C322ED
:10321A0078A3E630E21AAF728F70BF0204D22A8016
:10322A0002D22C7F04125783125719D214D22322A6
:10323A007899E6606916E670657811E214601814E8
:10324A00603B24027058633E0143390278117401CD
:10325A00F2789976148047E540C394EF400E7811CE
:10326A007402F24339027899761480327410254038
:10327A00F540D2044339027899760A8021E54070F4
:10328A000EF5404339027811F278997614800F745A
:10329A00F02540F540D2044339027899760AD22CB7
:0332AA00D223220A
:1032AD0078A4E630E70A7F027D6C123AB28F56227F
:1032BD0078A4E630E40A7F047D6C123AB28F562270
:1032CD0078A4E630E639E53330E1343032317B0530
:1032DD007A7079CAE4FD12540EE4FF12565FE4FFD2
:1032ED001256BC75701EE4F56CF54FF550C228C230
:1032FD0020D232D2307899F67880E24401F22278E9
:10330D00A4E630E253E530D394005007E56CD39436
:10331D007F4045E55630E0407F10D23A12575512A6
:10332D005719125737E4782EF2757035E53075F070
:10333D0064A47C00256CFFEC35F044C0F54F8F5034
:10334D00F573756C117880E24409F2D228C220D24F
:10335D0032C230789976022278A4E620E203023355
:10336D00E6E5307074E56C6070E55630E0347F1042
:10337D00D23A125755125719125737782E7405F243
:10338D00757035856C73754F00856C50756C017853
:10339D0080E24409F2D228C220D232C23078997626
:1033AD000222E55630E11C7570227880E24401F26C
:1033BD00856C6E756C01C228C220D232C230E478A1
:1033CD0099F622D207D20E856C6A75720175700559
:1033DD00781C7403F24339212278A4E630E54EE5DA
:1033ED0030704AE56C6046E55630E0237F10D23AE6
:1033FD00125755125719125737757020856C737502
:10340D006C017880E24409F2C230E47899F622E545
:10341D005630E1030236E6D207D20E856C6A75721C
:10342D0002757005433921781C7403F22278A3E6E6
:10343D0020E303023508303203023508E56C6012D3
:10344D00E53064096003023508E56C6450600302E1
:10345D003508E47886F2E53024F86045146064247C
:10346D000960030236E6E55630E02012571912576F
:10347D00377B057A7079C27D0112540EE4F573D253
:10348D00327880E24408F275702022D207D20EE421
:10349D00F56A757201757005433921781C7403F254
:1034AD00221257191257377562047850E55AF2E413
:1034BD00F55A782AF208F27842E24408F2C23075E1
:1034CD00702B22E56C7023757037782DF2D228C2DF
:1034DD002078A17463F278937402F2E4F56C782A83
:1034ED00F2D232C230433B04800375701D7F10D27F
:1034FD003A1257551257191257372278A3E630E36F
:10350D003F30323CE53320E1030236E67F10D23AFC
:10351D001257557B057A7079D6E4FD12540E125769
:10352D0019125737782E7409F2757035756C1D7830
:10353D0080E24405F2D228C220C230789976142256
:10354D0078A3E620E3030236D93032030236D9E5FB
:10355D003024FA70030236E61470030236E6147056
:10356D00030236181470030236472409600302362D
:10357D00C3E56CB4082212571912573775620478D7
:10358D0050E55AF2E4F55A782AF208F27842E2440C
:10359D0008F2D23075702B22E56CB409241257193C
:1035AD0012573778A17463F278937402F2E4F56CD4
:1035BD00782AF2782DF2D232433B04D2307570372F
:1035CD0022E56CC3946450030236E6E56CD3947324
:1035DD0040030236E675703B7F10D23A125755E420
:1035ED00FF12565FE4FF1256BC7B057A7079EEE44C
:1035FD00FD12540EE56C249C788EF2756C01C22878
:10360D00C220D232D230E47899F622E4F5607850B7
:10361D00E2FF655AFEF55AEF6EF2625A75702E1280
:10362D005719125737C228D220E4782AF27842E28D
:10363D004401F2C230E47899F622E56CC39450400F
:10364D0030E56CD3945C50297570177F10D23A1207
:10365D005755125719125737856C6AE56A54FC781D
:10366D0027F2E56A5403786AF2D228C220433B0858
:10367D0022E56CC394004061E56CD3943F505A75BC
:10368D0070387F10D23A125755E4FF12565FE4FF9F
:10369D001256BC7B057A7079EEE4FD12540E78A1BA
:1036AD00E56CF2756C01C228C220433B08D232D2C0
:1036BD0030E47899F622E530C39450401CE530D3C0
:1036CD00945650157866E2F56002361B7F6CD23A3F
:0A36DD001237F15004789976C822E4
:1036E700AE07EE30E0037F4022EE30E1037F802219
:0336F7007F00222F
:1036FA008F10E5107008125C098F10EF603A7FFF97
:10370A00125783125847123BC1123BA3123B9AC26B
:10371A001BC217E4F572757005786CE56AF2AF1092
:10372A008F3D8F6AE4F530F55630270778297404FF
:10373A00F28003433901D322E4F56AF53DF530F509
:03374A0056C32241
:10374D008F0F8D10E4F511E50F700F7F10125D6571
:10375D008F0F8F11EF70030237E4E51054E0FFBFB8
:10376D004011755E407880E24440F27572027570CA
:10377D00058047BF8018E50FC394415011755E80D9
:10378D007881E24440F2757202757005802CBF207D
:10379D0020E5116002150F755E207842E24404F2B7
:1037AD00E4782AF2756001757025F5727530088020
:1037BD00094339017572027570057FFF1257831227
:1037CD00586D123BC1786CE56AF2AF0F8F5A8F6A54
:1037DD00E4F564F530D322E4F55EF55AF56AF5307B
:0437ED00F556C322A8
:1037F1008F0FE4F510A807E6751100F512E5307595
:10380100F064A4AEF02512F512EE3511F51178A48D
:10381100E630E616303202C322AE11AF127C007DD3
:103821000A127B3F8E118F128032E4FF123B198FF7
:1038310010BFFF02C322AE11AF127C007D0A127BC2
:103841002BEF2510FFEC3EFEC3EF9512EE951150C4
:1038510007E4F511F51280048E118F12203A03024C
:1038610039A0AE11AF127C007D64127B3FEE600384
:10387100023938EFB40A004003023938903884F82D
:103881002828730238A20238A20238A20238E002C4
:1038910038EB0238F602390102398402390B023958
:1038A10084E55630E50BD3E5129463E5119400509D
:1038B10010E55630E410D3E5129450E51194004020
:1038C10005E4F511F512E55630E30ED3E512947FC8
:1038D100E51194004003023984E4F5300239A0E592
:1038E1005620E3030239A0023984E55620E303029E
:1038F10039A0023984E55620E3030239A002398454
:10390100E55620E3030239A08079C3E5129460E50E
:10391100119403501B74E02512F51274FC3511F556
:10392100117850E512F278667401F2753008806FF3
:10393100E55630E36A804CC3E5129440E511941FCB
:103941004031D3E51294BAE51194215026AE11AF5E
:10395100127C007D0A127B3FAF057866EFF2C394BB
:10396100014010E2FFD394045009E570B41A14EF3A
:10397100B40110C3E5129401E51194285021E556D4
:1039810030E31CAE11AF127C007D64127B3F8F309F
:10399100AE11AF127C007D64127B3F8C118D12D36E
:1039A100E51294FFE51194004007E4F530F511F5B7
:1039B1001230220AC222E53390719D93F5563032BE
:1039C1000AC232E4F530F511851012303A0EAF1209
:1039D100A80FEFF6FFAD301252AD800EAF12A80F57
:0C39E100EFF6FF7E007D041253A2D322FB
:1039ED008F0EA807E6FE08E68E0FF510E4F51178A8
:1039FD00A4E630E60FAF107C007D0A127B3F8E0FE0
:103A0D008F108020E4FF123B198F11BFFF02C322DC
:103A1D00AE0FAF107C007D0A127B2BEF2511F51038
:103A2D00EC3EF50F303208C232750F00851110D300
:103A3D00E51094E7E50F94034006750F008511100E
:103A4D00AE0FAF10A80EA60608A6077D041253A24E
:013A5D002246
:103A5E00AE07E53324FE601414601414601B14606A
:103A6E001B14602214602980007F00227F0922EE41
:103A7E0030E6037FA1227F00227F1222EE30E70381
:103A8E007F52227F0022EE30E7037F52227F0922EF
:103A9E00EE30E6037FA122EE30E7037F52227F0055
:043AAE00227F002251
:103AB2008D0F855610EF24FC6029240270567F403A
:103AC200123A5E8F10EF30E04BE55620E7107B058F
:103AD2007A7079F2E4FD12540E4310808030531054
:103AE2003E80207F80123A5E8F10EF30E626E55648
:103AF20020E60D7B057A7079F6E4FD12540E800EF5
:103B020053103D7B057A7079A6E4FD12540EC22251
:073B1200A80FE4F6AF10223A
:103B19008F1378A4E6FF30E10654FDF67F00227882
:103B2900A5E6F930E00654FEF67F0122E930E10806
:103B390054FD78A5F67F0222E930E20854FB78A506
:103B4900F67F0322E930E30854F778A5F67F0422CB
:103B5900E930E40854EF78A5F67F0522E930E50855
:103B690054DF78A5F67F0622E930E60854BF78A528
:103B7900F67F0722E930E70978A5E6547FF67F0842
:103B89002278A4E6FF30E00654FEF67F09227FFF83
:013B99002209
:093B9A00C218C208E478A2F62268
:103BA300E541554A6017E54154076003433902E58F
:0E3BB3004154386003433904E54AF45241227C
:103BC100E55C555D600DE55DF4525CE55B30E70356
:043BD100433908224A
:103BD50078A4E630E64EE57064017028E53F30E0F4
:103BE5000D20170AE4FF125F58125F07D22BAF6A48
:103BF500125CF2E4FF1236FA40057F0112277CE4DD
:103C0500F538801EE57064026005E570B42713126F
:103C15005E1CE4FFFD12374D40057F0112277CE451
:063C2500F555D322C32275
:103C2B00201B03301702C322300803023CD3E53EAE
:103C3B0030E503023CD3E53F540C24FC602924FC03
:103C4B00604424FC605D8000E540131313541FFF98
:103C5B00E536131313541FC39FFF127BE9D3EF6495
:103C6B0080948140638057E540131313541FFFE585
:103C7B0036131313541FC39FFF127BE9D3EF6480DA
:103C8B00948140448038E5401313543FFFE53613CD
:103C9B0013543FC39FFF127BE9D3EF6480948140A1
:103CAB0027801BC3E5369540FF127BE9D3EF648079
:103CBB009481500AE536B4010FE540B4020A85360B
:103CCB0040D204D223433902E53E30E520302607AB
:103CDB00E536D39402500A202613E536C3940250DE
:103CEB000C533EDFE478A2F6D22343390278A4E6E4
:103CFB0030E02A7871E220E724E5706403601EE56A
:103D0B0036C394025004D2268008C226D20878A269
:103D1B007646433E20E4F540C21843390278A2E6CA
:103D2B00FF7003023E5D127B943D650A3D6B143DB3
:103D3B0077163D8C183DA11A3DBA283DC0323DCCBB
:103D4B00343DE0363DF4383E0C463E1A503E25528B
:103D5B003E39543E4D5600003E5A125822023E5AEE
:103D6B007F177D02C23A1258BE023E5A7F17E4FDFE
:103D7B00C23A1258BE7F077D02C23A1258BE023EAB
:103D8B005A7F07E4FDC23A1258BE7F167D02C23A33
:103D9B001258BE023E5A7F16E4FDC23A1258BE7F3D
:103DAB00067D02C23A1258BE78A27607023E5A121C
:103DBB005822023E5A7F067D01C23A1258BE023E7D
:103DCB005A7F06E4FDC23A1258BE7F167D01C23AF5
:103DDB001258BE807A7F16E4FDC23A1258BE7F0796
:103DEB007D01C23A1258BE80667F07E4FDC23A12CB
:103DFB0058BE7F177D01C23A1258BE78A276258035
:103E0B004E1258227F067D02C23A1258BE80407F66
:103E1B00177D02C23A1258BE80357F17E4FDC23AB5
:103E2B001258BE7F077D02C23A1258BE80217F070F
:103E3B00E4FDC23A1258BE7F167D02C23A1258BE3A
:103E4B00800D7F16E4FDC23A1258BE78A2764378F5
:103E5B00A20678A3E6FF30E108633E01533EDF8004
:103E6B005DEF30E005633E08805478A4E630E44C07
:103E7B00E57064017046E53F6401F53F30E016AF35
:103E8B003D125F58AF3D125F137863E53DF2C22BD5
:103E9B00E4F538801EAF3D125EF0C22B125ECB8F65
:103EAB0010EF6005125C4F8002D22B7863E510F2A5
:103EBB00E4F538E47853F24339808002C322D223ED
:053ECB00433902D3227F
:103ED0007F14E53E30E3047D0280027D00D23A1279
:103EE00058BEE53E5411FF600464117026E53E3073
:103EF000E0047F0580027F157D03C23A1258BEE5BB
:103F00003E30E0047F1580027F05E4FDC23A12587E
:103F1000BE8024E53E30E0047F0580027F157D02EF
:103F2000C23A1258BEE53E30E0047F1580027F059C
:103F30007D01C23A1258BEE53F30E0137F80A217E0
:103F4000721B5003D38001C3923A12575580057FEC
:103F500080125783E5424543454545466006E55690
:103F6000540360077F0812578380077F08C23A1204
:103F7000575578A2E66003301B4B30040BC2047F18
:103F800006E4FDC23A1258BE7F173018047D028045
:103F9000027D00D23A1258BE7F07E53E30E108E5C7
:103FA0004860047D0380027D00C23A1258BE7F162D
:103FB000E53E30E208E54960047D0380027D00C2F1
:0E3FC0003A1258BE2278A2E6B4FF02E4F622BE
:103FCE00201B03301702C3227871E220E703024060
:103FDE0072E53F20E104D22CC3227F177D01C23A45
:103FEE001258BE78A5E6F930E009634E0254FEF68B
:103FFE0002424CE930E10B634E0454FD78A5F60203
:10400E00424CE930E20B634E0854FB78A5F60242AF
:10401E004CE930E30B634E1054F778A5F602424C90
:10402E00E930E40854EF78A5F6024248E930E50895
:10403E0054DF78A5F6024248E930E60854BF78A569
:10404E00F6024248E930E70978A5E6547FF60242C7
:10405E004878A4E6FF20E003024248634E0154FE76
:10406E00F602424C789BE630E7127F173018047D3B
:10407E000280027D00D23A1258BED22C78A5E6F903
:10408E007007789CE67002C322E54A30E0222007D2
:10409E001FE930E00B43410154FE78A5F602424C75
:1040AE00789CE6FF30E0185341FE54FEF602424C77
:1040BE00E930E00B63410154FE78A5F602424CE56F
:1040CE004A30E12220071FE930E10B43410254FD43
:1040DE0078A5F602424C789CE6FF30E1185341FD7C
:1040EE0054FDF602424CE930E10B63410254FD7877
:1040FE00A5F602424CE54A30E22220071FE930E2E3
:10410E000B43410454FB78A5F602424C789CE6FF23
:10411E0030E2185341FB54FBF602424CE930E20BFD
:10412E0063410454FB78A5F602424CE54A30E32283
:10413E0020071FE930E30B43410854F778A5F60238
:10414E00424C789CE6FF30E3185341F754F7F602E1
:10415E00424CE930E30B63410854F778A5F602426E
:10416E004CE54A30E42220071FE930E40B434110AE
:10417E0054EF78A5F602424C789CE6FF30E41853D3
:10418E0041EF54EFF602424CE930E40B6341105418
:10419E00EF78A5F602424CE54A30E5232007207859
:1041AE00A5E6FF30E50943412054DFF602424C7884
:1041BE009CE6FF30E5185341DF54DFF602424C789F
:1041CE00A5E6FF30E50863412054DFF68070E54A2E
:1041DE0030E62120071E78A5E6FF30E60843414071
:1041EE0054BFF68059789CE6FF30E6175341BF5412
:1041FE00BFF6804A78A5E6FF30E60863414054BF1B
:10420E00F6803BE54A30E72120071E78A5E6FF3011
:10421E00E708434180547FF68024789CE6FF30E720
:10422E001753417F547FF6801578A5E6FF30E708D7
:10423E00634180547FF68006C322D22CD3224339A9
:05424E0002D22CD32276
:104253007871E230E722E54E541FFFC313FF7D035D
:10426300E4FB1246317F01E54E30E0047D0380021A
:104273007D00C23A1258BE22AF417D03E4FB1246D1
:024283003122E6
:104285007828E2B40D004003024599904297F8283A
:1042950028730242BE0243DA0243E30243EC0243BF
:1042A500F50243FE02440702441002445A024473D5
:1042B5000244A002453502455678A4E630E326E5DA
:1042C50072640170207F04D23A1257557B057A70CB
:1042D50079FAE4FD12540EE4FF12565F7828740A49
:1042E500F2D206D32278A4E630E42CE5726401709C
:1042F50026755153F552F5537B047A007951FD1219
:10430500540E7F04D23A125755E4FF12565F7828AF
:10431500740BF2D206D32278A4E630E726E5726460
:104325000170207F04D23A1257557B057A7079F2D5
:10433500E4FD12540EE4FF12565F7828740CF2D295
:1043450006D322E4FF123B198F0FBFFF02C322AF32
:104355000F7828EFF27002C322E5726402702078AC
:1043650028E2FFB40705E55E30E714EF6408600F47
:10437500EFB40905E55E20E606E47828F2C322E5F8
:1043850072B4270B7828E264076004E4F2C322E5DF
:1043950072B40D06E47828F2C322E50F2430F551F6
:1043A500E4F552F5537B047A007951FD12540E7FE2
:1043B50004D23A125755E4FF12565FD2067828E226
:1043C50024FD600F240224FB500280077F08D23AA7
:1043D500125755D322751003750E4202459F75106D
:1043E50003750E4302459F75100F750E4802459FD4
:1043F500751007750E4502459F751003750E46022B
:10440500459F75100F750E4902459FE572B401046D
:104415007F4A80027F5D8F0EA807E6FF7D027B0144
:10442500124631E4FF123B198F0FEFF46025E50FBB
:104435006021A80EE6FFE50F90717E936FF6E57299
:10444500B40208A80EE6F4525C8006A80EE6F45203
:1044550041D322C322E572B402047F5980027F3C16
:104465008F0E7510097861E24402F202459FE572EC
:10447500B4010975100F750E4702459FE55E54019D
:10448500F50F7F0F7D011245AC4002C322E50F7089
:1044950005535EFE8003435E01D322750E4BA80EC5
:1044A500E6FF1246E6E4FF123B198F0FEFF47003A7
:1044B500024533EF24FE602514603D146055240346
:1044C500706AA80EE6FF30E40554EEF6805EEF3024
:1044D500E0054410F68055EF4401F6804FA80EE63E
:1044E500FF30E50554DDF68043EF30E1054420F665
:1044F500803AEF4402F68034A80EE6FF30E6055414
:10450500BBF68028EF30E2054440F6801FEF4404F7
:10451500F68019A80EE6FF30E7055477F6800DEF13
:1045250030E3054480F68004EF4408F6D322C32225
:10453500E53F5430FFC4540FF50F7F0F7D02124540
:10454500AC4002C322533FCFE50FC454F0423FD3E2
:10455500227F03E53F30E1047D0180027D02C23AFE
:104565001258BE7F13E54E30E7047D0180027D02BF
:10457500C23A1258BEE4FF123B198F0FEFF46012D6
:10458500EF24FE600804700A633F02D322634E8065
:10459500D322C322E47828F2C322AF0EAD10124510
:0745A500AC4002C322D32247
:1045AC008F118D12A807E6FF12514A7B047A00790D
:1045BC0051E4FD12540EE4FF123B19EFF4603E304F
:1045CC000612EFD395125006A811A607802BA8113E
:1045DC00E4F68025E512D394094014A811E675F091
:1045EC000AA42FF6D395124010A811E4F6800AEF16
:1045FC00D395125004A811A607C206801478A4E61D
:10460C0030E60CC206A811E675F00A84F6D322C374
:10461C0022A811E6FF12514A7B047A007951E4FD7D
:05462C0012540ED32220
:104631008F118D128B137F03E51130E004AE1280D0
:1046410004AE13AD06C23A1258BE7F13E51130E134
:1046510006AE12AD068004AE13AD06C23A1258BEC4
:104661007F04E51130E206AE12AD068004AE13AD53
:1046710006C23A1258BE7F11E51130E306AE12AD03
:10468100068004AE13AD06C23A1258BE7F02E51190
:1046910030E406AE12AD068004AE13AD06C23A1286
:1046A10058BE7F12E51130E506AE12AD068004AEAC
:1046B10013AD06C23A1258BEE4FFE51130E606AE6C
:1046C10012AD068004AE13AD06C23A1258BE7F1079
:1046D100E51130E706AE12AD068004AE13AD06C299
:0546E1003A1258BE2250
:1046E6008F11E51120E005E4F512800DE51130E4A7
:1046F6000575120280037512017F03AD12C23A12CC
:1047060058BEE51120E105E4F512800DE51130E50E
:104716000575120280037512017F13AD12C23A129B
:1047260058BEE51120E205E4F512800DE51130E6EC
:104736000575120280037512017F04AD12C23A128A
:1047460058BEE51120E305E4F512800DE51130E7CA
:104756000575120280037512017F11AD12C23A125D
:0347660058BE2218
:10476900AE5DE47869F278A5E6F97007789CE670A1
:1047790002FF22E55E54C06011E55E30E1037F026D
:1047890022E55E30E70F7EFF800BE55B7007E56091
:1047990020E702E4FEEE30E02220071FE930E00BBB
:1047A900435C0154FE78A5F6024978789CE6FF300F
:1047B900E018535CFE54FEF6024978E930E00B63D9
:1047C9005C0154FE78A5F6024978EE30E122200713
:1047D9001FE930E10B435C0254FD78A5F6024973E9
:1047E900789CE6FF30E118535CFD54FDF6024973ED
:1047F900E930E10B635C0254FD78A5F6024973EEDA
:1048090030E22220071FE930E20B435C0454FB78B5
:10481900A5F602496E789CE6FF30E218535CFB541A
:10482900FBF602496EE930E20B635C0454FB78A5A0
:10483900F602496EEE30E32220071FE930E30B430D
:104849005C0854F778A5F6024969789CE6FF30E3DD
:1048590018535CF754F7F6024969E930E30B635CD6
:104869000854F778A5F6024969E55E5441FFBF414E
:10487900037F0022EE30E42320072078A5E6FF30ED
:10488900E409435C1054EFF6024964789CE6FF3072
:10489900E419535CEF54EFF602496478A5E6FF305A
:1048A900E409635C1054EFF6024964EE30E5232015
:1048B900072078A5E6FF30E509435C2054DFF602BE
:1048C900495F789CE6FF30E518535CDF54DFF60258
:1048D900495F78A5E6FF30E508635C2054DFF68080
:1048E90075EE30E62120071E78A5E6FF30E608437D
:1048F9005C4054BFF6805A789CE6FF30E617535C5B
:10490900BF54BFF6804B78A5E6FF30E608635C40EC
:1049190054BFF6803CEE30E72120071E78A5E6FF5C
:1049290030E708435C80547FF68021789CE6FF30AD
:10493900E717535C7F547FF6801278A5E6FF30E7CE
:1049490008635C80547FF680037F00227869E20463
:10495900F27869E204F27869E204F27869E204F231
:104969007869E204F27869E204F27869E204F27F94
:02497900012219
:10497B00E55E30E67930E06C7F03E55F30E1047D86
:10498B000180027D02C23A1258BE7F13E55F30E30D
:10499B00047D0180027D02C23A1258BE7F04E55F9E
:1049AB0030E5047D0180027D02C23A1258BE7F11B0
:1049BB00E55F30E7047D0180027D02C23A1258BEEA
:1049CB007F02E4FDC23A1258BE7F12E4FDC23A12D6
:1049DB0058BEE4FFFDC23A1258BE7F10E4FDC23A46
:1049EB001258BE22AF5F7D03E4FB12463122E55E17
:1049FB0030E70AAF5F7D017B0212463122AF5C7D4F
:074A0B00017B02124631227B
:104A1200750C01750D02E55F655CF50EE56030E72A
:104A220008750C03E4F50DF50EE56330E00B7F032A
:104A32007D04C23A1258BE801F7F03E55C30E00657
:104A4200AE0CAD068004AE0DAD06E50E30E003D32C
:104A52008001C3923A1258BEE56330E10B7F137DA9
:104A620004C23A1258BE801F7F13E55C30E106AEE5
:104A72000CAD068004AE0DAD06E50E30E103D38029
:104A820001C3923A1258BEE56330E20B7F047D0403
:104A9200C23A1258BE801F7F04E55C30E206AE0CBB
:104AA200AD068004AE0DAD06E50E30E203D3800103
:104AB200C3923A1258BEE56330E30B7F117D04C204
:104AC2003A1258BE801F7F11E55C30E306AE0CAD92
:104AD200068004AE0DAD06E50E30E303D38001C3BC
:104AE200923A1258BEE56330E40B7F027D04C23A6B
:104AF2001258BE801F7F02E55C30E406AE0CAD06A4
:104B02008004AE0DAD06E50E30E403D38001C392FE
:104B12003A1258BEE56330E50B7F127D04C23A12A9
:104B220058BE801F7F12E55C30E506AE0CAD0680F4
:104B320004AE0DAD06E50E30E503D38001C3923A13
:104B42001258BEE56330E60BE4FF7D04C23A125808
:104B5200BE801FE4FFE55C30E606AE0CAD068004C5
:104B6200AE0DAD06E50E30E603D38001C3923A12D4
:104B720058BEE56330E70A7F107D04C23A1258BE80
:104B8200227F10E55C30E706AE0CAD068004AE0D68
:104B9200AD06E50E30E703D38001C3923A1258BE48
:014BA20022F0
:104BA300E4F5C04390075390C7E52CF4F52CF5C00A
:104BB300D293E52DF4F52DF5C0D294C293E52EF4EE
:104BC300F52EF5C0D293E52FF4F52FF5C0D293D28D
:104BD30094D295B213A212B39212500820200B5311
:104BE30090EF80062028035390E7E4F5C05390F834
:104BF300E537429075C0FFE5375403FFE5C0F4FE87
:104C0300E4F5C05390F8EF7008E5C430E2034306BF
:104C130008748F2FF8E25EFDEEF274702FF8E2FE57
:104C230074A32FF8EEF45D46F6749A2FF8EDF45E54
:104C330046F674702FF8EDF20537E537D394064046
:104C430003753704E5C520E403024D0B53C5EF7824
:104C53008BE224FE602114605424026003024D059C
:104C630085C636301806E536C313F53675C509789B
:104C73008B7402F2024D1BE5C6C39450500FE5C678
:104C8300D394054008E531600D15318009E531C342
:104C9300940A50020531E5C6C394055003D380013D
:104CA300C3922975C508788B7403F2806BAFC6EF86
:104CB3002535F535E43534F5347894E204F2C394BC
:104CC300084035E4F2E535AE347803CEC313CE1392
:104CD300D8F9F5358E34F56BE4F534F535AFC6EF19
:104CE3002567F567E43566F566789D06E67009E5A0
:104CF30066F571E4F566F56775C50F788B7401F297
:104D03008016E4788BF28010788BE2700BE5C55443
:104D130018700575C50F04F230083AE540C4540F06
:104D2300FFE536C4540F6F702C78A276FFC208D209
:104D3300237F067D03C23A1258BE7F177D03C23A12
:104D43001258BE7F077D03C23A1258BE7F167D03F9
:064D5300C23A1258BE2214
:104D5900E532700A0528E528B40303E4F5285390E1
:104D6900F8E5324290E4F5C0301F19E52830E00A31
:104D790074B02532F8E6F5C0802174802532F8E652
:104D8900F5C08017E52830E00A749E2532F8E6F56B
:104D9900C08008747A2532F8E6F5C0E53204540378
:034DA900F53222BE
:104DAC00E4F50C7473250CF8E2540F14601D1460B8
:104DBC002A1460371460442404704EE50C907191F1
:104DCC0093FF7D02C23A1258BE803EE50C90719161
:104DDC0093FF7D05C23A1258BE802EE50C9071915E
:104DEC0093FF7D06C23A1258BE801EE50C9071915D
:104DFC0093FF7D01C23A1258BE800EE50C90719162
:104E0C0093FF7D07D23A1258BE050CE50CC39408EB
:104E1C0040917839E2F50C6044E4F2E50C54072437
:104E2C0031F551E50C30E508755255755345801A2E
:104E3C00E50C30E3047F4280027F2D8F52E50C306D
:104E4C00E4047F4280027F2D8F53E4F5547F0212DD
:0E4E5C00565F7B047A0079517D0212540E22BB
:104E6A007871E230E4087864EFF2433B8022E5701F
:104E7A00B40F06786EE26F70437841EFF22473F84C
:104E8A00E2540FFE7899E6C3940A50160EE570B400
:104E9A000F04BE04010EEED394044002E4FEE4784B
:104EAA0099F6E570B40F08EE44807864F2800478CD
:0D4EBA0064EEF2433B0274952FF8E4F222FF
:104EC70078A1E2FFAD301252AD12586D788AE254E4
:104ED7000F1460211460321460431460542404706A
:104EE70062786EE290719193FF7D02C23A1258BECA
:104EF700750C48804E786EE290719193FF7D05C2E4
:104F07003A1258BE750C55803A786EE290719193BB
:104F1700FF7D06C23A1258BE750C4C8026786EE2A9
:104F270090719193FF7D01C23A1258BE750C46806D
:104F370012786EE290719193FF7D07D23A1258BEB4
:104F4700750C41786EE22431F55175522D75532D4C
:104F57007812E230E5087552557553458011788A05
:104F6700E2FF30E403850C52EF30E503850C53E490
:104F7700F5547F0212565F7B047A0079517D021245
:034F8700540E22A3
:104F8A007884E230E71CE4F50CE50C90719193FF0C
:104F9A007D02D23A1258BE050CE50CC3940940E9C9
:104FAA0080487882E2F50DE4F50CAF0CAD0D125095
:104FBA0024E50D1313543FF50D050CE50CC39404B9
:104FCA0040E87883E2F50DE50CC394085013AF0C62
:104FDA00AD0D125024E50D1313543FF50D050C8049
:104FEA00E67F087884E2FD125024D220C22878A1F4
:104FFA00E2FFAD301252AD7884E230E60B7B057ADF
:10500A007079FE7D0212540E7884E230E50B7B053E
:0A501A007A7079D27D0212540E2242
:105024008F0EED54031460191460251460312403A9
:10503400703BE50E90719193FF7D01C23A1258BE08
:1050440022E50E90719193FF7D03C23A1258BE225D
:10505400E50E90719193FF7D03D23A1258BE22E57A
:0E5064000E90719193FF7D04C23A1258BE2245
:10507200788DEFF27871E230E606788DE24440F204
:105082007899E6B40A06788DE24480F27860E244C8
:0350920020F222E7
:1050950012586D789AE230E21DE4F50CE50C90713A
:1050A5009193FF7D02D23A1258BE050CE50CC394CC
:1050B5000840E9D21422786AE2F50E750D01E4F58F
:1050C5000CE50CC3940850227495250EF8E2550D95
:1050D500600EE50C90719193FF7D02C23A1258BEA5
:1050E500050CE50D25E0F50D80D77862E2FFF4604B
:1050F50027EF131313541FFE786AE2B506047E01E9
:1051050080027E00EE5403600FEF54079071919377
:10511500FF7D01D23A1258BE7899E2FF131313545A
:105125001FFE786AE2B506047E0180027E00EE5419
:1051350003600FEF540790719193FF7D01C23A12FE
:0551450058BED2142247
:10514A00EF75F00A84E5F02430F553EF75F00A8420
:10515A00FF75F00A84E5F02430F552B43003755235
:02516A00202201
:10516C00E538F46033E53824F6601B8000E538241C
:10517C0020FF74052538FD7B021273274003025271
:10518C00AC05380538227F2B7D3A7B011272F0403A
:10519C00030252AC7538FF22E555F4606BE55524DB
:1051AC00F660538000E555C3940A5025E55524302C
:1051BC00FF741D2555FD7B0212732740030252AC70
:1051CC00E5552402F555640A60030252AC7555107E
:1051DC0022E5552440FF74462555FD7B02127327AA
:1051EC0040030252ACE5552402F555641A600302E3
:1051FC0052AC75550A227F3B7D587B011272F040F0
:10520C00030252AC7555FF227861E230E023E4F5DD
:10521C000D301B03430D01E570B40103430D027FF8
:10522C00027D0D7B011272F050767861E254FEF231
:10523C00227861E230E125E572B40108853C0D75F8
:10524C000C03800685590D750C04AF0C7D0D7B018C
:10525C001272F0504B7861E254FDF2227861E23028
:10526C00E21D750E5A750F417F067E0EAD067B0250
:10527C001272F0502B7861E254FBF24408F222785F
:10528C0061E230E31BAF8A786DEFF2F50E7F087E9A
:10529C000EAD067B011272F050067861E254F7F203
:0152AC0022DF
:1052AD008D13EFFD7C00E51375F064A4AEF02DF5C4
:1052BD0015EC3EF514FEAF157D0A127B3FED243043
:1052CD00F553AE14AF157C007D0A127B3F8E148F03
:1052DD00157C007D0A127B3FED2430F552AE14AFE4
:1052ED00157C007D0A127B3F8E148F157C007D0A84
:1052FD00127B3FED2430F551E55630E70575514CE5
:10530D008019E55630E60575514F800FE551B430E3
:10531D0012E513C3940A500B755120E552B43003B6
:10532D00755220301B12E570B4010D7B047A0079A3
:10533D00517D0112540E800B7B047A007951E4FDEE
:10534D0012540EE513C3940A404AAE14AF157C00F7
:10535D007D0A127B3F8E148F157C007D0A127B3FD8
:10536D00ED2430F553AE14AF157C007D0A127B3F52
:10537D008E148F157C007D0A127B3FED2430F55283
:10538D00B430037552207551207B047A0079517D1C
:05539D000612540E226F
:1053A2008D13AB07AA067C007D0A127B3FED2430E9
:1053B200F553AE02AF037C007D0A127B3FAA06AB17
:1053C200077C007D0A127B3FED2430F552AE02AF1E
:1053D200037C007D0A127B3FAA06AB077C007D0A94
:1053E200127B3FED2430F551E51330E210E551B464
:1053F200300B755120E552B430037552207B047A8C
:0C540200007951E5135403FD12540E22F2
:10540E008B168A178918EDB40700400302563290A6
:10541E005424F82828730254390254920254F40288
:10542E00553B0255790255B70255F5AB16AA17A989
:10543E0018127AE190710293FF783DE25480FEEFEC
:10544E004EF27843F27847F2784BF2900001127ADE
:10545E00FC90710293FF783EE25480FEEF4EF2789C
:10546E0044F27848F2784CF2900002127AFC907175
:10547E000293783FF27845F27849F2784DF27FFF49
:10548E001257A222AB16AA17A918127AE19071022E
:10549E0093FF783DE25480FEEF4EF27843F2900097
:1054AE0001127AFC90710293FF783EE25480FEEF77
:1054BE004EF27844F2900002127AFC9071029378C8
:1054CE003FF27845F27847E25480F2784BF2784812
:1054DE00E25480F2784CF27849E25480F2784DF240
:1054EE007FFF1257A222AB16AA17A918127AE190C3
:1054FE00710293FF7847E25480FEEF4EF2784BF242
:10550E00900001127AFC90710293FF7848E2548069
:10551E00FEEF4EF2784CF2900002127AFC9071027D
:10552E00937849F2784DF27FFF1257A222AB16AA5A
:10553E0017A918127AE190710293FF783DE2548018
:10554E00FEEF4EF2900001127AFC90710293FF78FA
:10555E003EE25480FEEF4EF2900002127AFC907101
:10556E000293783FF2E4FF1257A222AB16AA17A9B4
:10557E0018127AE190710293FF7843E25480FEEFA5
:10558E004EF2900001127AFC90710293FF7844E281
:10559E005480FEEF4EF2900002127AFC907102934C
:1055AE007845F27F011257A222AB16AA17A918123C
:1055BE007AE190710293FF7847E25480FEEF4EF24B
:1055CE00900001127AFC90710293FF7848E25480A9
:1055DE00FEEF4EF2900002127AFC9071029378491F
:1055EE00F27F021257A222AB16AA17A918127AE15D
:1055FE0090710293FF784BE25480FEEF4EF29000D2
:10560E0001127AFC90710293FF784CE25480FEEF07
:10561E004EF2900002127AFC90710293784DF27F56
:05562E00031257A22247
:10563300783DE27843F27847F2784BF2783EE278AD
:1056430044F27848F2784CF2783FE2FF7845F2FF73
:0C5653007849F2784DF27FFF1257A22236
:10565F00EF1460211460382402704C783DE24480CE
:10566F00F27843E24480F27847E24480F2784BE2EA
:10567F004480F28032783DE24480F27843E2448005
:10568F00F27847E2547FF2784BE2547FF280187839
:10569F003DE2547FF27843E2547FF27847E2448050
:0D56AF00F2784BE24480F27FFF1257A222F6
:1056BC00EF1460211460382402704C783EE2448070
:1056CC00F27844E24480F27848E24480F2784CE28A
:1056DC004480F28032783EE24480F27844E24480A6
:1056EC00F27848E2547FF2784CE2547FF2801878DA
:1056FC003EE2547FF27844E2547FF27848E24480F0
:0D570C00F2784CE24480F27FFF1257A22297
:10571900783DE2547FF27843E2547FF27847E254CD
:0E5729007FF2784BE2547FF27FFF1257A222EC
:10573700783EE2547FF27844E2547FF27848E254AC
:0E5747007FF2784CE2547FF27FFF1257A222CD
:105755007840E24FF27846E24FF2303A11784AE269
:10576500FEEFF4FDEE5DF2784EE25DF2800A784AD6
:0E577500E24FF2784EE24FF27FFF1257A2226F
:105783007840E2FEEFF4FDEE5DF27846E25DF278FA
:0F5793004AE25DF2784EE25DF27FFF1257A222EA
:1057A200C2A9BFFF077884E6FEFF8000EF14601FE6
:1057B20014603114604324037054783DE2F52C08E0
:1057C200E2F52D783FE2F52E7840E2F52F803F7822
:1057D20043E2F52C08E2F52D7845E2F52E7846E213
:1057E200F52F802A7847E2F52C08E2F52D7849E278
:1057F200F52E784AE2F52F8015784BE2F52C08E277
:10580200F52D784DE2F52E784EE2F52FB2163013D3
:105812000C632CFF632DFF632EFF632FFFD2A9229F
:105822007F17E4FDC23A1258BE7F07E4FDC23A1266
:1058320058BE7F16E4FDC23A1258BE7F06E4FDC28E
:055842003A1258BE22DD
:10584700E478B3F618F618F618F678A1F618F618ED
:10585700F618F67883F618F618F618F6787DF6181F
:06586700F618F618F62207
:10586D007F03E4FDC23A1258BE7F13E4FDC23A1223
:10587D0058BE7F04E4FDC23A1258BE7F11E4FDC24A
:10588D003A1258BE7F02E4FDC23A1258BE7F12E4AE
:10589D00FDC23A1258BEE4FFFDC23A1258BE7F1047
:1058AD00E4FDC23A1258BE7F01E4FDC23A1258BE61
:0158BD0022C8
:1058BE00EF131313541FFEEF540790717F93FFEDF8
:1058CE00B409004003025C089058DDF828287302E2
:1058DE0058F802593902598A0259DB025A38025ACB
:1058EE0075025AD4025B33025B9674B02EF8EFF455
:1058FE0056F674B12EF8EFF456F6749E2EF8EFF4B9
:10590E0056F6749F2EF8EFF456F674802EF8EFF4D8
:10591E0056F674812EF8EFF456F6747A2EF8EFF4EC
:10592E0056F6747B2EF8EFF456F62274B02EF8E687
:10593E004FF674B12EF8EFF456F6749F2EF8EFF47E
:10594E0056F674802EF8E64FF674812EF8EFF45664
:10595E00F6747B2EF8EFF456F6303A11749E2EF84C
:10596E00EFF456F6747A2EF8EFF456F622749E2E55
:10597E00F8E64FF6747A2EF8E64FF62274B12EF84A
:10598E00E64FF674B02EF8EFF456F6749E2EF8EF3E
:10599E00F456F674812EF8E64FF674802EF8EFF476
:1059AE0056F6747A2EF8EFF456F6303A11749F2E9E
:1059BE00F8EFF456F6747B2EF8EFF456F622749F39
:1059CE002EF8E64FF6747B2EF8E64FF62274B02EC4
:1059DE00F8E64FF674B12EF8E64FF674802EF8E620
:1059EE004FF674812EF8E64FF6303A21749E2EF85B
:1059FE00EFF456F6749F2EF8EFF456F6747A2EF8EE
:105A0E00EFF456F6747B2EF8EFF456F622749E2EB3
:105A1E00F8E64FF6749F2EF8E64FF6747A2EF8E6F7
:105A2E004FF6747B2EF8E64FF62274B02EF8E64F42
:105A3E00F674B12EF8EFF456F6749E2EF8EFF45677
:105A4E00F6749F2EF8E64FF674802EF8E64FF67435
:105A5E00812EF8EFF456F6747A2EF8EFF456F674AB
:105A6E007B2EF8E64FF62274B02EF8E64FF674B1A0
:105A7E002EF8E64FF674802EF8EFF456F674812E5B
:105A8E00F8E64FF6303A21749E2EF8EFF456F6747F
:105A9E009F2EF8EFF456F6747A2EF8EFF456F6744D
:105AAE007B2EF8EFF456F622749E2EF8E64FF6741F
:105ABE009F2EF8E64FF6747A2EF8EFF456F6747BB6
:105ACE002EF8E64FF62274B02EF8E64FF674B12E8D
:105ADE00F8E64FF674802EF8E64FF674812EF8EF46
:105AEE00F456F6303A21749E2EF8EFF456F6749F63
:105AFE002EF8EFF456F6747A2EF8EFF456F6747B11
:105B0E002EF8EFF456F622749E2EF8E64FF6749F9A
:105B1E002EF8E64FF6747A2EF8E64FF6747B2EF8D2
:105B2E00EFF456F62274B02EF8EFF456F674B12E4A
:105B3E00F8EFF456F674802EF8EFF456F674812EC4
:105B4E00F8E64FF6303A21749E2EF8EFF456F674BE
:105B5E009F2EF8EFF456F6747A2EF8EFF456F6748C
:105B6E007B2EF8EFF456F622749E2EF8EFF456F6CE
:105B7E00749F2EF8EFF456F6747A2EF8EFF456F66C
:105B8E00747B2EF8E64FF62274B02EF8E64FF674BC
:105B9E00B12EF8EFF456F6749F2EF8EFF456F67415
:105BAE00802EF8EFF456F674812EF8EFF456F67454
:105BBE007B2EF8EFF456F6303A21749E2EF8EFF461
:105BCE0056F6749F2EF8EFF456F6747A2EF8EFF41C
:105BDE0056F6747B2EF8EFF456F622749E2EF8E6E7
:105BEE004FF6749F2EF8EFF456F6747A2EF8EFF403
:0B5BFE0056F6747B2EF8EFF456F622EA
:105C0900202B1A125ECB8F12EF60107863E26512B7
:105C19006001227405253AF8E512F2D22BE4F51158
:105C2900E511D3953C501CE53A04FFE4FDAB3C1269
:105C39005F908F3A74052FF8E2F5126002FF220592
:065C49001180DD7F002246
:105C4F008F11E511606C125CC38F12EFF460058544
:105C5F00123AC322E4F512E512D3953C5021E53AEE
:105C6F0014FFE4FDAB3C125F908F3A74052FF8E2FE
:105C7F00700974052FF8E511F2D322051280D8E4CC
:105C8F00F512E512D3953C5027E53A14FFE4FDAB2E
:105C9F003C125F908F3A74052FF8E2FF125E89BFB6
:105CAF00FF0A7405253AF8E511F2D322051280D2C6
:045CBF00C322C32217
:105CC3008F13E4F514853A15E514D3953C501D74F0
:105CD300052515F8E2B51303AF1522E51504FFE416
:0F5CE300FDAB3C125F908F15051480DC7FFF2214
:105CF2007EFFE4FD74052DF8E2B50704E4F2AE057B
:075D02000DBD0AF0AF0622FF
:105D0900E4FF74052FF8E2FE6006653D6002C322D8
:065D19000FBF0AEED322C9
:105D1F00E4FFEFD3953C500C74052FF8E27002C3EB
:065D2F00220F80EED322DA
:105D3500AC077BFFE4FA74142AF8E2FF6009125CF1
:105D4500F2EFF46002AB070ABA08EBEBF4600BAFB5
:105D5500038F3A74052FF8ECF222AF04125C4F2240
:105D65008F12E4F513E55804FFE4FDAB59125F907B
:105D75008F58741D2FF8E2FF600A74562558F8E213
:105D8500A812F6220513E513C3940A40D87F002212
:105D95008F0E8D0FE50E6045125DE48F10EFF460F8
:105DA50005851058C322E4F510E55814FFE4FDAB52
:105DB50059125F908F58741D2FF8E26005E510B5F4
:105DC5005912741D2558F8E50EF274562558F8E554
:0F5DD5000FF2D3220510E510C3940A40CCC3226D
:105DE4008F118D12E4F513855814741D2514F8E2EF
:105DF400B5110C74562514F8E2B51203AF1422E55C
:105E04001404FFE4FDAB59125F908F140513E513DE
:085E1400C3940A40D57FFF2270
:0F5E1C0074562558F8E4F2741D2558F8E4F22264
:105E2B00C23AE4FE741D2EF8E2B5071674562EF82E
:105E3B00E2B5050E741D2EF8E4F274562EF8E4F25A
:095E4B00D23A0EBE0ADEA23A2290
:105E5400E4FFFEEED39559500B741D2EF8E2600159
:0F5E64000F0E80EFEFD394014003C38001D322D0
:105E7300E4FFEFD39559500C741D2FF8E27002C361
:065E8300220F80EED32285
:105E89008F19E5196028E4F51A85571B7414251B29
:105E9900F8E2B51903AF1B22E51B04FFE4FD7B07FC
:105EA900125F908F1B051AE51AC3940840DE7FFF25
:015EB90022C6
:105EBA00E4FF74142FF8E26002C3220FBF08F3D381
:015ECA0022B5
:105ECB00E4F513E55704FFE4FD7B07125F908F5752
:105EDB0074142FF8E2FF6001220513E513C3940835
:055EEB0040E17F0022F0
:105EF000C23AE4FE74142EF8E2B50704E4F2D23A92
:075F00000EBE08F0A23A22D8
:0C5F0700E4FF7F087814E4F208DFFC22BD
:105F13008F11E511603D125E898F12EFF4600585E4
:105F23001257C322E4F512E55704FFE4FD7B071281
:105F33005F908F5774142FF8E26005E512B4070AD7
:105F430074142557F8E511F2D3220512E512C39410
:055F53000840D4C32248
:105F5800AC07E4FB74142BF8E2FF60066C600312D4
:075F68005CF20BBB08EE2206
:105F6F00AE07C3ED6480F8EE6480985003AF05224E
:105F7F00D3EB6480F8EE6480984003AF0322AF0642
:015F8F0022EF
:105F9000AE07C3ED6480F8EE6480985003AF03222F
:105FA000D3EB6480F8EE6480984003AF0522AF061F
:015FB00022CE
:105FB100EFC39D5002C322EFD39B4002C322D322E1
:0F5FC100E4FEEF20E0060EC313FF80F6AF0622CA
:105FD000EF1FAC0670011E4C6012301AFDC21A3061
:0D5FE0002DEEC22D43871075FF3280E422A4
:075FED00AE071FEE70FA225F
:105FF4007F011272E47F437D1C7B1A1271FA7FFFCA
:106004007DFF12723F7FC01272DB7F221272E42284
:10601400C2AD303B02D21E7529C81272DEEF30E2E7
:106024000E7F8F12728F7FC11272DBD2ADD322D555
:0660340029E8D2ADC322F1
:10603A00C2AD300002D21E752A141272DEEF30E2AF
:10604A0010C2197FA612728F7FC11272DBD2ADD332
:08605A0022D52AE6D2ADC322D3
:10606200783BE539F27852E53BF27842E27851F238
:106072007880E27885F27881E27887F27860E27857
:1060820065F2202708A23A923B12601422A23A92A9
:05609200021260AC22C7
:10609700D219302708A20192021260AC22A2019203
:0560A7000012603A2226
:1060AC00300202D21E12746350103019097F8F7D9A
:0C60BC00A67B0A127A3EC219D322D3221E
:1060C8007885E624E5B436004003026C329060DC43
:1060D800F828287302617E02617E026C32026C32FB
:1060E800026C32026FB102621D0262A70262D9021B
:1060F8006337026FB1026FB1026FB1026FB1026F05
:10610800B1026FB1026FB1026FB1026FB1026FB12C
:10611800026FB102635902646B0264EC02652F02DC
:10612800665002672C026AA9026B07026B52026F63
:10613800B1026FB1026FB1026FB1026FB1026FB1FC
:10614800026FB1026FB102621D0262A70262D90238
:106158006337026FB1026FB1026FB1026FB1026FA4
:10616800B1026FB1026FB1026FB1026FB1026FB1CC
:10617800026FB1026B8EE570640D6009E570640B07
:106188006003026FB17887E6656A6003026FB178D1
:1061980086E6FFC4135407F51CC394084003026F36
:1061A800B1E570B40B0C7495251CF8E220E70302E6
:1061B8006FB17888E6FF7473251CF8EFF2D20522D8
:1061C8007887E6FFB55A21E570B4021C78A67634C4
:1061D80008760408A607087601786DE278AAF6E43E
:1061E80008F6C201126097227887E6FF125E89EFEF
:1061F800F47003026FB178A676340876047887E6DF
:1062080078A8F6087602786DE278AAF6E408F6C26D
:1062180001126097227887E6FF653D702AE5706075
:106228002664056022201B1F78A6763408760408A9
:10623800A607E408F6786DE278AAF6E53F54E00888
:10624800F6C201126097227887E6FFB55A24E570F6
:10625800B4021F78A6763408760408A607087601E3
:10626800786DE278AAF6E55E54E008F6C20112609D
:1062780097227887E6FF125E89EFF47003026FB108
:1062880078A676340876047887E678A8F608760241
:10629800786DE278AAF6E408F6C20112609722E562
:1062A8003D7887666003026FB1E5706401600302A0
:1062B8006FB1201B03026FB108E6F53E08E6F53F13
:1062C80008E6F54008E6F54108E6F54ED223D22C5B
:1062D80022E53D7887666003026FB1E5706401606E
:1062E80003026FB1201B03026FB108E6F54108E60F
:1062F800FFC4540FF542EF540FF54308E6FFC454AA
:106308000FF544EF540FF54508E6FFC4540FF54662
:10631800EF540FF54708E6FFC4540FF548EF540F44
:10632800F54908E6F54A08E6F54BD223D22C22E5D2
:106338005A7887666003026FB1E5706402600302F1
:106348006FB108E6F55B08E6F55C08E6F55DD22A6C
:10635800227886E6FF30E504787F7640201E030227
:106368006FB1E57064056003026FB1EF540F640507
:10637800703A788BE624FC5008602014601D026F88
:10638800B1E54C7887666003026FB1E54D08666039
:1063980003026FB175703675723622E56A788766C2
:1063A8006003026FB175703675723622E54C54C0C1
:1063B80064C07026E54C788C66701FE54D086670E1
:1063C800197887E6F56AF53D08E6F53E08E6F53FF3
:1063D80008E6F54008E6F541806BE53390719D933A
:1063E80030E32BE56AD3947F40247887E6FF656A1B
:1063F800701C8F3D08E6F53E08E6F53F08E6F540D7
:1064080008E6F54108E6F54C08E6F54D803778874B
:10641800E6FF656A6003026FB18F3D08E6F53E0846
:10642800E6F53F08E6F54008E6F54108E6FFC454FE
:106438000FF542EF540FF54308E6FFC4540FF54437
:10644800EF540FF545787FE60479A6F7E53D540744
:10645800FFC43354E0440178A7F608A63DD20112E0
:10646800609722E53D7887666003026FB1E5706446
:10647800056003026FB1201E03026FB108E6FFC476
:10648800540FF546EF540FF54708E6FFC4540FF5CF
:1064980048EF540FF54908E6F54A08E6F54B08E6D3
:1064A800F54E20253A75701B757201E53F30E02DD9
:1064B800302B057863E53DF2125EBA500A43398005
:1064C80078537401F28018AF3D125E898F1CEFF487
:1064D8006007851C57C22B8006D2178002D22BC2B8
:1064E8001EC225227886E630E504787F76407887D4
:1064F800E6FF656A6003026FB1E570640560030238
:106508006FB1201E03026FB18F5A08E6F55B08E6EB
:10651800F55C08E6F55DE4F55E20240675701C75EB
:106528007202C21EC224227886E6540F24FE604FEF
:1065380014607414602614606E24046003026FB142
:106548007887E6FF653D6011EF655A6003026FB119
:10655800E55E54C06003026FB1C21E22788AE6FF6E
:10656800600C64026008EF64016003026FB1E53DEE
:106578007887666003026FB175703675723622E5EA
:106588005A7888666003026FB118E6FF30E205E5C5
:106598005E20E70FEF30E203026FB1E55E20E6030D
:1065A800026FB1435E0222E55A7888666003026F83
:1065B800B118E6FF30E217E55E30E712755E8078C5
:1065C80089E6F55FF55CE4F55D535EFD8058EF30D4
:1065D800E203026FB1E55E20E603026FB1EF5401FA
:1065E80065646003026FB1755E417889E6FFF55F07
:1065F80008E6F55D535EFD08E630E007535EFE8F62
:106608005C8023E4F55CE55F30E103435C01E55F12
:1066180030E303435C02E55F30E503435C04E55F78
:1066280030E703435C08E570B4050975701C7572A2
:1066380002C21E22E57064026009E570640360030B
:10664800026FB1D22AC21E22E570700302670D30B4
:106658000A0630270302670BE56A7887666003023B
:106668006702AF6A125E89EFF46003125F077888E9
:10667800E6FF702AD21BD223D22CD21478A2F6E5D8
:10668800726402600302670BE55E54E07075D22401
:1066980075720175700543390175650A8065EF6487
:1066A800017023788AE654E0701CE5726401705327
:1066B800E53F54E0704DD225757202757005433977
:1066C8000175650A803DEF64027038E572B4010E09
:1066D800D21BD223D22CD214E478A2F68025E572FC
:1066E8006402701FE55E54E07019D224757201755A
:1066F800700543390175650A8009E53D788766703C
:1067080002D21BC20A7887E6FF125E89EFF4700393
:10671800026FB1AF3D125E89EFF46004D21BD21450
:10672800125F07227887E6127B94676C00678701FF
:1067380067A80267D20367E10467F205682806685C
:106748003D07695C0869B70969D60A69E40B69EC11
:106758000C69FB0D69FE0E6A0A146A66176A7018DE
:1067680000006FB1E47868F2C20CE5706427600538
:10677800E572B4270475702922857270D2142278C4
:1067880068E2FF64016002D216EF6406600578686B
:106798007401F2200C057899760A22E47899F62299
:1067A800E57064207003026FB1E570642470030221
:1067B8006FB17868E2FF64036002D216EF64077075
:1067C80003026FB178687403F2227868E2640260A9
:1067D80002D21678687402F222E53D788866600372
:1067E800026FB108E6F53ED22322E57064207003FB
:1067F800026FB1E57064357003026FB1E57064240F
:106808007003026FB1E57064056008757009C21EF7
:10681800E4F53978687404F2C219E4F53BC236220B
:10682800E57064206003026FB17888E6FF7E00E4BB
:10683800FD1253A222E570B4201B7889E6FF7E0082
:10684800E4FD1253A27F10C23A1257557889E6F533
:106858007375701F22E57064356003026FB1782E7E
:10686800E2B40E004003026FB1906878F8282873EC
:106878000268A20268B40268C30268D9026FB10252
:1068880068DF0268EE026904026FB102690A0269F0
:106898002E026942026FB1026951855073756C12FC
:1068A8007880E24408F2782EE204F222756C1D78B2
:1068B80080E24404F2782EE204F2227889E6442049
:1068C800F573756C1D7880E24408F2782EE204F2C4
:1068D80022782EE204F222756C1D7880E24404F2DC
:1068E800782EE204F2227889E654DFF573756C1D80
:1068F8007880E24408F2782EE204F222782EE2044C
:10690800F2227889E630E50F756C127880E244044B
:10691800F2782EE204F222756C017880E24404F2E7
:10692800782E740DF2227889E6F573756C117880EB
:10693800E24404F2782EE204F2227889E6F54FE583
:1069480073F550782EE204F2227889E6F573782EF2
:10695800E204F222E5706420702578857645087691
:10696800527888E624307987F77B017A0079857D2B
:106978000112540E7F10C23A12575575701F22E546
:106988007064356003026FB1788576450876527871
:1069980088E624307987F77B017A0079857D0112B2
:1069A800540E7F10C23A125755782E74FFF222E522
:1069B8003D7888666003026FB1E53F54307003028A
:1069C8006FB17810E26003026FB1740AF222E53DFC
:0A69D8007888666003026FB1781042
:1069E200F2227888E65407F533227868E26405607B
:1069F20002D21678687405F222120000E57064244F
:106A02006003026FB1D23022E57064317026E53D39
:106A1200788866701F7F20125783782AE2D39420E9
:106A22005003026FB17F10C23A125755757030E4AD
:106A3200782AF222E57064346003026FB17888E646
:106A42006003026FB17F20125783782AE2D3942029
:106A52005003026FB17F10C23A125755757033E47A
:106A6200782AF222E57064316003026FB1227886DF
:106A7200E6540F64076003026FB17889E61460067A
:106A8200046003026FB1E570643D6003026FB17F81
:106A920010C23A125755788DE6FF7E00E4FD12537C
:106AA200A275703CC21E22E53D7887666003026FC4
:106AB200B1E57064056003026FB1201E03026FB17D
:106AC20008E6FFC4540FF546EF540FF54708E6FFFA
:106AD200C4540FF548EF540FF54908E6F54A08E6A5
:106AE200F54B08E6F54E20250675701B757201C23E
:106AF2001EE53F30E0047F0280027F007888A6070F
:106B0200C22502666078A1E2788766700CE570643F
:106B1200106018E57064126012788BE620E70302B9
:106B22006FB1E57064026003026FB17888E678A104
:106B3200F27889E67882F2788AE67883F2788BE6D0
:106B42007884F2E570B41003757011D209C21E2266
:106B5200E53D7887666003026FB1301B03026FB1B7
:106B6200301703026FB1F51C7487251CF8E6FF7419
:106B720014251CF8EFF2051CE51CB408EB7863E55C
:106B82003DF2C22BC217D223E4F557227827E2FF47
:106B92007887666008EF64506003026FB17888E618
:106BA200FF0846FE08E6FD4EFE08E6FC4E700302B4
:106BB2006FB17886E654E0FE6480703EE57064143E
:106BC2006006E570641670327895EFF27889E6789F
:106BD20096F27897EDF27898ECF2788CE6600116EE
:106BE200788CE67899F2788DE6789AF2E570B414AA
:106BF20006757015757215D20F22EE6003026FB121
:106C0200E57064166003026FB17889E66001167858
:106C120089E6FF7899F2EF131313541F5403FF7898
:106C22006AF27827E22FF56A789A7401F2D20F227B
:106C32007885E654C064C06003026D6408E6FF54C0
:106C4200E06440703BEF540F64027034E570B43A74
:106C5200187F10C23A1257557888E6FF7E00E4FD8D
:106C62001253A2757039C21E22E5706437600302A6
:106C72006FB1782DE204F27888E6543F79A1F322CD
:106C82007886E6FF54E064206003026FB1EF540F90
:106C920064087003026FB17885E6543FFF656A604D
:106CA20009E56A64636003026FB17887E6F51CC385
:106CB20094084003026FB1E570640B70377888E680
:106CC200FE7495251CF8EEF27889E6FE7473251C95
:106CD200F8EEF2E4F51C7495251CF8E220E70302B5
:106CE2006FB1051CE51CB408ED75700C75720CD201
:106CF20005C21E22E570640D702A7495251CF8E207
:106D02007888666011E6FE7495251CF8EEF2EE5462
:106D1200B8451C7839F27889E6FE7473251CF8EEC2
:106D2200F2D20522E570640F6003026FB17889E642
:106D3200FE5430700818E620E503026FB178A1EF27
:106D4200F2786EE51CF27888E6FF7812F2749525E7
:106D52001CF8EFF2788AEEF27473251CF8EEF2D288
:106D620010227885E6FF54C064806003026FB10888
:106D7200E6FE7010E570B42B0B782BE204F2EF54B0
:106D82003FF55A22EF543F655A6003026FB1EE5449
:106D9200E0FF64A06005EF64207072E57064276014
:106DA20006E57064267066E56030E7617887E6FE86
:106DB200131313541F540304FEE56030E6047D01EF
:106DC20080027D00C3EE9DF51CE560540F651C60DA
:106DD20003026FB17887E6FE5407F51C9071889321
:106DE2005263EE30E50AE51C90717F934263801A8C
:106DF200EE30E60CE51C90717F93425F425C800AA4
:106E0200E51C90718893525F525CD20B22EF706D39
:106E12007887E67045E570642E703F7850E55AF247
:106E22007866E560F2E55A75F00AA4FF7888E67C98
:106E3200002FFFEC35F0FEE4FD1253A2E4FF1256E0
:106E4200BC1257197F10C23A1257557F02D23A121A
:106E52005755C228C22075702C227887E6B4011BD0
:106E6200E570B42E167F10C23A1257557889E6FFA4
:106E72007E00E4FD1253A275702D22C21E7886E6B2
:106E820054E0FF6420706008E6FEC4540F540124ED
:106E920001FDE433FCE560540F6D7001EC7048E5D0
:106EA2007064276006E5706426703C7887E6FE54BD
:106EB2000FFDC313F51C907188935263EE30E50AFF
:106EC200E51C90717F934263801AEE30E60CE51C5C
:106ED20090717F93425F425C800AE51C90718893B7
:106EE200525F525CD20B22EF64406003026FB1E545
:106EF2007064256003026FB17886E6540FF6E4F5FC
:106F02005DF55BE560540FF56024FE602214604F6E
:106F120014607124036003026F997886E6B4080353
:106F22004360807887E6F55D788BE6F55F80687868
:106F320086E6FFB4080A4360807888E6F55D80182B
:106F4200EFB4070A4360C07889E6F55D800AEF6412
:106F52000670537889E6F55D788CE6F55F803878BF
:106F620086E6FFB4080A4360807889E6F55D800D05
:106F7200EF640770314360C0788AE6F55D788DE68C
:106F8200F55F80137886E6B4081C436080788AE651
:106F9200F55D788EE6F55F855F5CE4F563755E20EE
:106FA200757026C21E22757028E4782AF2C21E224B
:03000B00026FB2CF
:106FB200C0E0C0F0C083C082C0D0C000C001C00227
:106FC200C003C004C005C006C007C28C758CFD7525
:106FD2008A65D28CA203B392035002D21A30B20B4A
:106FE200E56FC394FF5007056F8003E4F56F052B2F
:106FF200E52B24FC6015146028240324FA50352460
:1070020007702630272EE4F5C08029124D59301C16
:1070120008C293D294D295801BD293D294D29580F7
:1070220013302710E4F5C0800B124BA3124D59E424
:10703200F52BD22DD007D006D005D004D003D00234
:0F704200D001D000D0D0D082D083D0F0D0E032B7
:03002B000270510F
:10705100C0E0C0F0C083C082C0D0C000C001C00287
:10706100C003C004C005C006C007C2AD1272E1EF83
:1070710030E00D7F851272BF7FC41272DB1260C8CF
:10708100D2ADD007D006D005D004D003D002D001B4
:0D709100D000D0D0D082D083D0F0D0E0323B
:1071FA0078A2EFF208EDF208EBF21272EA78A5EF44
:10720A00F220E007E24401FF1272E47F0678A2E26C
:10721A00FD1272D17F0778A3E2FD1272D17F08783E
:10722A00A4E2FD1272D17F017D801272D178A5E2AB
:05723A00FF1272E422C6
:10723F0078A2EFF208EDF21272EA78A4EFF220E0F2
:10724F0007E24401FF1272E47F0478A2E2FD12729A
:10725F00D17F0578A3E2FD1272D178A4E2FF1272FA
:02726F00E42217
:10727100ED601AEF4420F5DB0BEBAE0270010A144E
:0E728100F5828E83E0F5DAAF051DEF70EB228B
:10728F00A2AF9233C2AF8FD875DB8A0000A23392C0
:02729F00AF221C
:1072A100ED601AEF4420F5DB0BEBAE0270010A141E
:0E72B100F5828E83E5DAF0AF051DEF70EB225B
:1072BF00A2AF9234C2AF8FD875DB940000A2349284
:0272CF00AF22EC
:0572D1008FDB8DDA22C5
:0572D6008FDBAFDA229E
:0372DB008FD92226
:0372DE00AFD82204
:0372E100AFD92200
:0672E400E4F5DB8FDA2265
:0672EA00E4F5DBAFDA223F
:1072F0008F108D118B12C23A1273E87FA012740B9B
:10730000501FAF1012740B5018D23AAF121512EF73
:10731000600FAF110511A807E6FF12740B40ECC215
:077320003A1273F8A23A22B1
:107327008F108D118B12C23A1273E87FA012740B63
:10733700501FAF1012740B5018D23AAF121512EF3C
:10734700600FAF110511A807E2FF12740B40ECC2E2
:077357003A1273F8A23A227A
:10735E008F0C8D0D8B0EC23A1273E87FA012740B38
:10736E00502DAF0C12740B50261273E87FA11274BD
:10737E000B501CD23AAF0E150EEF6013E50E24FF24
:10738E00923B127430AE0D050DA806A60780E612CC
:05739E0073F8A23A2281
:1073A3008F0C8D0D8B0EC23A1273E87FA012740BF3
:1073B300502DAF0C12740B50261273E87FA1127478
:1073C3000B501CD23AAF0E150EEF6013E50E24FFDF
:1073D300923B127430AE0D050DA806EFF280E61253
:0573E30073F8A23A223C
:1073E800C2AFD2B000D2B100C2B000C2B1D2AF2297
:1073F8007F64C2B100C2B000D2B100D2B020B002E6
:03740800DFF02290
:10740B007E08C2AFEF3392B0EF25E0FFD2B100C2DE
:10741B00B1DEF1D2B000D2B100A2B0B3923BC2B197
:05742B00D2AFA23B22DC
:107430007F08C2AFD2B0E4FED2B100A2B0E43342C2
:1074400006C2B1EFD394014004EE25E0FEDFE9303F
:107450003B03C38001D392B000D2B100C2B1D2AF1E
:03746000AF062252
:10746300D236E577700A30A807E56FC3943C500223
:10747300C322C28E53890F438910758DFF758B9B71
:0C748300D28EC2A8C28FD2ABD2B6D322E8
:0300030002748FF5
:10748F00C0E020B226E570602230271FC28E5389DC
:10749F000F438910758DFF758B0AD28EC28FD2ABB9
:1074AF00C2A8D237E577700375770CE4F56FD0E09B
:0174BF00329A
:03001B000274C0AC
:1074C000C0E0C083C082C0D0C000C006C007C28E6A
:1074D000E577B4170040030279D79074E1F82828C3
:1074E000730275260275500275660275800275A5D5
:1074F0000275C30275D30275F702762D0276420239
:10750000765802766C02769B0276B20276DB0276C1
:10751000F902770F0277320277490277A6027804E0
:1075200002782D0279BE20B70B758DFD758B65D263
:107530008E0279FD20B209C2ABC289D2A80279FDC0
:10754000758DFA758BCAD28ED2B57577010279FD29
:10755000758D97758BDBD28EC2B5757702C289D2D5
:10756000A8C2B60279FD758DFD758B65D28E30B2DD
:10757000030276852037030276857577030279FD4D
:1075800030B203027685758DE5758BF6D28E7890D4
:10759000E6540F2402F57675748F757501757704BE
:1075A000D2B60279FD20B70B758DFD758B65D28E35
:1075B0000279FDC2B5758DFD758BCFD28E757705BD
:1075C0000279FDD2B5758DFE758B63D28E75770607
:1075D0000279FDA874E6557524FFB392B5500A757B
:1075E0008DFE758B63D28E8008758DFD758BCFD225
:1075F0008E7577070279FDA2B5B392B5500A758DE5
:10760000FE758B63D28E8008758DFD758BCFD28E03
:10761000E5752575F575700FD576067577090279CC
:10762000FD7577080279FD7577060279FDC2B5759B
:107630008DF5758B95D28E0574757501757704027D
:1076400079FD758D97758BDBD28E75770AC2B5C2C1
:1076500089D2A8C2B60279FD758DF8758B2FD28EAE
:1076600020B22230371F75770B0279FD20B216E564
:107670008A541F2432F565E4F577C236C2ABC2895D
:10768000D2A80279FDE4F577E58A541F2432F56526
:10769000C2ABC289D2A8C2B60279FD758DFE758BC8
:1076A000B2D28E30B2030279EA75780875770D028E
:1076B00079FD758DFE758BB2D28E30B2030279EAF8
:1076C0001578E57860030279FDC28E758DE5758BBE
:1076D000F6D28E75770ED2B60279FD20B70B758D76
:1076E000FD758B65D28E0279FDD2B5758DFA758BDD
:1076F000CAD28E75770F0279FDC2B5758D97758BDD
:10770000DBD28E757710C289D2A8C2B60279FD7518
:107710008DFE758B15D28E30B2030279EA203703C5
:107720000279EA75748575760C75750175771102A5
:1077300079FD758DFE758B15D28E30B20675771278
:107740000279FD7577130279FD758DFE758B15D263
:107750008E30B2030279EAA874E64575F6E5752520
:1077600075F575703BE576B40B097886E6540FF530
:10777000766007AF761576EF7012C28E758DE5755F
:107780008BF6D28E757715D2B60279FDC28E758DC5
:10779000E5758BF6D28E757714C289D2A80279FD71
:1077A0007577110279FD758DFE758B15D28E20B21D
:1077B000030279EAA874E575F456F6E5752575F5C2
:1077C00075703BE576B40B097886E6540FF5766064
:1077D00007AF761576EF7012C28E758DE5758BF654
:1077E000D28E757715D2B60279FDC28E758DE5758C
:1077F0008BF6D28E757714C289D2A80279FD75777F
:10780000110279FD758DFE758B15D28E30B2030293
:1078100079EA2037030279EA0574E574D3948E403F
:10782000030279EA7575017577110279FD7885E6AD
:10783000FF24E5B436004003027995907842F82899
:1078400028730278E40278E4027995027995027946
:10785000950279EA0279EA0278F902790602791347
:107860000279EA0279EA0279EA0279EA0279EA021D
:1078700079EA0279EA0279EA0279200279EA027960
:10788000EA02792D0279470279510279A202795BE5
:107890000279A202796B02797402797E0279EA0296
:1078A00079EA0279EA0279EA0279EA0279EA027966
:1078B000EA0279EA0279EA0278F902790602791392
:1078C0000279EA0279EA0279EA0279EA0279EA02BD
:1078D00079EA0279EA0279EA0279200279EA027900
:1078E000EA027987E570640D70030279A2E570649D
:1078F0000B70030279A20279EAE53D78876670038E
:107900000279A20279EAE53D78876670030279A2DE
:107910000279EAE55A78876670030279A20279EA69
:10792000E55A78876670030279A20279EAE54C7815
:107930008C667009E54D086670030279A2E56A78E5
:107940008766605E0279EAE53D7887666054027971
:10795000EAE56A788766604A0279EA7887E6FE6532
:107960006A603FE53D6E603A0279EAE53D788766F8
:107970006030807678A1E27887666026806CE53D8D
:10798000788766601D8063E57064166015E5706435
:1079900014600F8055EF54C0FF64806005EF64C031
:1079A000704820B70A758DFD758B65D28E804ED2DA
:1079B000B5758DF5758B95D28E757716803FD2355E
:1079C000E4F577E58A541F2432F565C2B5C2ABC22F
:1079D00089D2A8C2B68026C2ABC289D2A8E58A5491
:1079E0001F2432F565E4F5778013E4F577E58A54D2
:1079F0001F2432F565C2ABC289D2A8C2B6C237D045
:0E7A000007D006D000D0D0D082D083D0E032A4
:107A0E008E838F828D01E709F0A3DBFA228C838DA2
:107A1E00828F01E0F709A3DBFA228F008D01E3F6D6
:107A2E000809DBFA228F008D01E7F20809DBFA2242
:0B7A3E008F008D01E7F60809DBFA223B
:03000000027A4938
:107A490078FFE4F6D8FD75A00078007F00E4F2081D
:087A5900DFFC7581B3027A9C89
:107A6100020100E493A3F8E493A34003F68001F23A
:107A710008DFF48029E493A3F85407240CC8C33326
:107A8100C4540F4420C8834004F456800146F6DFF5
:107A9100E4800B01020408102040809071E1E47E33
:107AA100019360BCA3FF543F30E509541FFEE493EA
:107AB100A360010ECF54C025E060A840B8E493A3B1
:107AC100FAE493A3F8E493A3C8C582C8CAC583CADC
:107AD100F0A3C8C582C8CAC583CADFE9DEE780BE94
:0171F9000095
:107AE100BB020689828A83E0224003BB0402E722AB
:0B7AF100400789828A83E49322E3228D
:107AFC00BB020CE58229F582E5833AF583E022404E
:107B0C0003BB0406E92582F8E622400DE58229F53F
:0F7B1C0082E5833AF583E49322E92582F8E22299
:107B2B00EFF88DF0A4FFEDC5F0CEA42EFEEC88F09F
:047B3B00A42EFE2254
:107B3F00BC000BBE0029EF8DF084FFADF022E4CC2A
:107B4F00F875F008EF2FFFEE33FEEC33FCEE9DECF3
:107B5F00984005FCEE9DFE0FD5F0E9E4CEFD22ED39
:107B6F00F8F5F0EE8420D21CFEADF075F008EF2F83
:107B7F00FFED33FD4007985006D5F0F222C398FD74
:057B8F000FD5F0EA2211
:107B9400D083D082F8E4937012740193700DA3A380
:107BA40093F8740193F5828883E473740293686094
:067BB400EFA3A3A380DF94
:0F7BE900C3EF6480948040028004EFF404FF2215
:107BBA00EF4E6013EDBB021089828A83EF60010EDB
:107BCA00EDF0A3DFFCDEFA2289F04003BB0407F7DD
:0F7BDA0009DFFCA9F02250EFF309DFFCA9F0222C
:00000001FF
